:020000040000FA
:0600000091EF39F012003F
:0600080086EF22F0120059
:0600180022EF00F01200CF
:06002A00020070730000EB
:1000300000050000E70000006E730000B90E00002C
:0400400002000000BA
:0C004400D8CFE4FFE0CFE4FFE46EDACF99
:10005000E4FFE2CFDAFFE9CFE4FFEACFE4FFF6CF37
:10006000E4FFF7CFE4FFF5CFE4FFF3CFE4FFF4CFF5
:10007000E4FFFACFE4FF00EE31F0140EE80403E3EE
:10008000EECFE4FFFBD700EE45F0090EE80403E3F2
:10009000EECFE4FFFBD7E652D9CFE6FFE1CFD9FFA1
:1000A000040EE126020EDB6A030EDB6AA4A650D31F
:1000B000A49605011B511C1104E005011B07000E4D
:1000C0001C5B05011D511E1104E005011D07000EFA
:1000D0001E5B0E01002B0E01AB510E01005D01E213
:1000E000B2D10E01006B0E01A951EA6A310FE96E1F
:1000F0000E0EEA22EF500E01EA6AAC25E96EAD5110
:10010000EA22EF6A79907B6A7A6A0E01A92B0E01C6
:10011000AA510E01A95D02E30E01A96B0E01A951BE
:10012000E96EEA6AD890E936EA36010EE9260E0E43
:10013000EA22EE50ED1001E186D10E01A951E96EDF
:10014000EA6AD890E936EA36490EE9260E0EEA2226
:10015000EECF4EF0EFCF4FF00E01A951E96EEA6AF3
:10016000D890E936EA36010EE9260E0EEA22EECFE5
:1001700050F0EFCF51F050504E1802E151504F184F
:1001800001E113D10E01A951E96EEA6AD890E9366E
:10019000EA36790EE9260E0EEA22EE50ED101FE146
:1001A0000E01A951E96EEA6AD890E936EA36490E9D
:1001B000E9260E0EEA22EECF4EF0EFCF4FF00E0101
:1001C000A951E96EEA6AD890E936EA36010EE926C5
:1001D0000E0EEA224EC0EEFF4FC0EDFFE6D00E013C
:1001E000A951E96EEA6AD890E936EA36490EE9265D
:1001F0000E0EEA22EECF50F0EFCF51F00E01A951D2
:10020000E96EEA6AD890E936EA36010EE9260E0E62
:10021000EA22EE50505C4E6EEE5051584F6E020E78
:100220004EC0DBFF030E4FC0DBFF020EDBCF4EF0F4
:10023000030EDBCF4FF04F3404E24E500008000EA7
:100240004F5458E2020EDBCF4EF0030EDBCF4FF0DF
:100250000E01A951E96EEA6AD890E936EA36790EBC
:10026000E9260E0EEA22EECF50F0EFCF51F04E50BD
:10027000505C4F5051581FE20E01A951E96EEA6AD5
:10028000D890E936EA36790EE9260E0EEA22EECF4C
:100290004EF0EFCF4FF00E01A951E96EEA6AD89007
:1002A000E936EA36010EE9260E0EEA224E50EE2617
:1002B0004F50ED221ED00E01A951E96EEA6AD89086
:1002C000E936EA36490EE9260E0EEA22EECF4EF066
:1002D000EFCF4FF00E01A951E96EEA6AD890E936E6
:1002E000EA36010EE9260E0EEA224EC0EEFF4FC09E
:1002F000EDFF5BD0020EDBCF4EF0030EDBCF4FF0F5
:100300004E6C4F1E000E4F220E01A951E96EEA6A93
:10031000D890E936EA36790EE9260E0EEA22EECFBB
:1003200050F0EFCF51F04E50505C4F5051581FE2FB
:100330000E01A951E96EEA6AD890E936EA36790EDB
:10034000E9260E0EEA22EECF4EF0EFCF4FF00E016F
:10035000A951E96EEA6AD890E936EA36010EE92633
:100360000E0EEA224E50EE5E4F50ED5A1ED00E0198
:10037000A951E96EEA6AD890E936EA36490EE926CB
:100380000E0EEA22EECF4EF0EFCF4FF00E01A95144
:10039000E96EEA6AD890E936EA36010EE9260E0ED1
:1003A000EA224EC0EEFF4FC0EDFF0E01A951EA6AEE
:1003B000310FE96E0E0EEA22EF500E01EA6AAC250B
:1003C000E96EAD51EA22120EEF6EF29EE66A0E0160
:1003D000A951EA6A310FE96E0E0EEA22EF50E66E7D
:1003E00095EC17F0E552E5520E01A951E96EEA6A63
:1003F000D890E936EA36010EE9260E0EEA22EECF53
:100400004EF0EFCF4FF04FC04EF04F6A4E50B66EE9
:100410000E01A951E96EEA6AD890E936EA36010E72
:10042000E9260E0EEA22EECF4EF0EFCF4FF04E50FF
:10043000B56EF00EB4140009B46EF00EB4140909D0
:10044000B46E7980F28E000ED8801D54000E1E54BA
:100450002EE22C2A000E2D221D502C5C1E502D58F1
:1004600026E32C6A2D6A030E215C1FE21F50EA6A04
:10047000480FE96E010EEA2280CFEFFF1F50EA6AB3
:100480004B0FE96E010EEA2281CFEFFF1F50EA6A9F
:100490004E0FE96E010EEA2282CFEFFF1F2A030EF4
:1004A0001F5C01E31F6A212A02D01D6A1E6A000E2A
:1004B000D8802254000E235419E22750000816E277
:1004C0002E2A000E2F2222502E5C23502F580EE38E
:1004D0002E6A2F6A030E265C07E2242A030E245C90
:1004E00001E3246A262A02D0226A236A27500008E0
:1004F0000AE2306A3050040DF328C26E9E9C9F9C25
:100500009D8CC280C2820501005101E11CD1DE6ACE
:10051000DD6ADECF4EF0DDCF4FF0040E4E5C000EF4
:100520004F5801E310D1DECFE9FFDDCFEAFF010E26
:10053000D890E936EA36E806FBE1010EE926050E19
:10054000EA22EE50ED1001E1D3D0DECFE9FFDDCF9E
:10055000EAFF010ED890E936EA36E806FBE1110E13
:10056000E926050EEA22EE50ED1026E1D9CFE9FF8B
:10057000DACFEAFFEE50ED1001E18180D9CFE9FF3B
:10058000DACFEAFF010EEE1801E1ED5001E18182C0
:10059000D9CFE9FFDACFEAFF020EEE1801E1ED5004
:1005A00001E18184D9CFE9FFDACFEAFF030EEE182B
:1005B00001E1ED5001E18186DECFE9FFDDCFEAFF09
:1005C000010ED890E936EA36E806FBE1110EE9267D
:1005D000050EEA22EECF4EF0EFCF4FF0DECFE9FF6F
:1005E000DDCFEAFF010ED890E936EA36E806FBE1F6
:1005F000010EE926050EEA22EECF50F0EFCF51F0C2
:1006000050504E1802E151504F1826E1D9CFE9FF62
:10061000DACFEAFFEE50ED1001E18190D9CFE9FF8A
:10062000DACFEAFF010EEE1801E1ED5001E181920F
:10063000D9CFE9FFDACFEAFF020EEE1801E1ED5063
:1006400001E18194D9CFE9FFDACFEAFF030EEE187A
:1006500001E1ED5001E18196DECFE9FFDDCFEAFF58
:10066000010ED890E936EA36E806FBE1110EE926DC
:10067000050EEA22EE2A000EEF22DECFE9FFDDCFE3
:10068000EAFF010ED890E936EA36E806FBE1110EE2
:10069000E926050EEA22EECF4EF0EFCF4FF0DECF87
:1006A000E9FFDDCFEAFF010ED890E936EA36E80629
:1006B000FBE1090EE926050EEA22EECF50F0EFCF5E
:1006C00051F050504E1802E151504F1810E1DECF5A
:1006D000E9FFDDCFEAFF010ED890E936EA36E806F9
:1006E000FBE1110EE926050EEA22EE6AED6A26D03C
:1006F000D9CFE9FFDACFEAFFEE50ED1001E18190AA
:10070000D9CFE9FFDACFEAFF010EEE1801E1ED5093
:1007100001E18192D9CFE9FFDACFEAFF020EEE18AC
:1007200001E1ED5001E18194D9CFE9FFDACFEAFF91
:10073000030EEE1801E1ED5001E18196DF2A010E72
:1007400001E3DB2AE6D60101F15102E00101F107E4
:100750009EAC2DD09E9CC450526E52C053F0526A33
:10076000C35000015210506E53C051F03050060D6E
:10077000F3CF4EF0F4CF4FF0000E4E26010E4F2275
:100780002450020D4E50F324E96E4F50F420EA6ECF
:1007900050C0EEFF51C0EDFF302A2750305C02E31D
:1007A0009D9C05D03050040DF328C26EC282F2A485
:1007B00042D0D59EF294F29A040E4E6E2B50EA6A05
:1007C000510FE96E010EEA22EF504E5C34E1080E43
:1007D0002B5C0DE2070E2B144E6E010E4E5204E000
:1007E000E846FE0B4E06FCE1E81C89161CD0100EF4
:1007F0002B5C0DE2070E2B144E6E010E4E5204E0E0
:10080000E846FE0B4E06FCE1E81C8A160CD0070EEB
:100810002B144E6E010E4E5204E0E846FE0B4E06BF
:10082000FCE1E81C8B162B50EA6A510FE96E010EB1
:10083000EA22020EEF6E040EE15C02E2E16AE5528A
:10084000E16EE552E7CFD9FFE55200EE4DF0090E1B
:10085000E80403E3E5CFEDFFFBD700EE44F0140E10
:10086000E80403E3E5CFEDFFFBD7E5CFFAFFE5CFE3
:10087000F4FFE5CFF3FFE5CFF5FFE5CFF7FFE5CFD9
:10088000F6FFE5CFEAFFE5CFE9FFE5CFDAFFE55078
:10089000E5CFE0FFE5CFD8FF1000D9CFE6FFE1CFED
:1008A000D9FF020EE126896A9268276A8A6A9368EC
:1008B0008B6A94688C968C9495969594928E06018A
:1008C000010EFD6F0E01B969BA69256A246A266AAC
:1008D000206A1F6A216A1D6A1E6A226A236A2C6ABC
:1008E0002D6A2E6A2F6A306A76827680769C769A96
:1008F00076887696FA0E776EDF6ADFCF45F00C0EBB
:10090000E76E4518E8AE02D0E73402D0E750455C08
:1009100038E2010EDB6A010EDBCF45F0030EE76E15
:100920004518E8AE02D0E73402D0E750455C27E234
:10093000DFCF45F0466A45BE4668060E4602F3CF55
:1009400046F0060E4502F3CF45F0F4504626000E61
:100950004526010E4622010EDBCF47F0486A47BE0E
:100960004868D8904736483645504724E96E465087
:100970004820EA6EEE6AED6A010EDB2ACCD7DF2A48
:10098000BCD70601F76B0601F86B0601F56B060193
:10099000F66B0601F96B0601FA6B0601FB6B0601AB
:1009A000FC6B296A2A6A2B6ADF6ADFCF45F0180ED2
:1009B000E76E4518E8AE02D0E73402D0E750455C58
:1009C0001BE2DFCFE9FFEA6AE9BEEA68D890E936C0
:1009D000EA36690EE926010EEA22EE6AED6ADFCFF9
:1009E000E9FFEA6AE9BEEA68510EE926010EEA2249
:1009F000010EEF6EDF2AD9D7D586D59AD59CF29411
:100A0000F29AF194D08E7694A386A5961EEC24F0EB
:100A100076EC33F0F28EF28C768493849392000E0F
:100A2000E66EE66A000EE66EE66A030EE66E000EFD
:100A3000E66EE66AABEC34F0456E070EE15E4550BB
:100A40000501196B0501D00E1B6F070E1C6F9396E5
:100A50008196020EE15C02E2E16AE552E16EE55246
:100A6000E7CFD9FF1200D9CFE6FFE1CFD9FF050EBE
:100A7000E126020EDB6A030EDB6A040EDB6AEEEC93
:100A800016F005011951040A01E17FD0070A75E04B
:100A9000010A41E0030A21E0010A01E092D00501C8
:100AA0001B511C1119E1200EE66ED10EE66E000EF0
:100AB000E66EE66AD00EE66E070EE66E1CEC26F0D9
:100AC000456E060EE15E45500501B80E1B6F0B0E1C
:100AD0001C6F0501010E196F75D005011B511C110A
:100AE00019E1000EE66EE66A000EE66EE66A030E97
:100AF000E66EF00EE66E550EE66EABEC34F0456E2B
:100B0000070EE15E4550640E05011B6F1C6B05016D
:100B1000020E196F57D005011B511C112DE1815098
:100B2000040B2AE1000EE66EE66A000EE66EE66A47
:100B3000030EE66E000EE66EE66AABEC34F0456E30
:100B4000070EE15E4550100EE66E270EE66E000EB3
:100B5000E66EE66AD00EE66E070EE66E1CEC26F038
:100B6000456E060EE15E45500501B80E1B6F0B0E7B
:100B70001C6F0501030E196F25D005011B511C11B7
:100B800003E10501040E196F1DD081A419D0F00EE8
:100B9000E66ED80EE66E000EE66EE66AD00EE66EE3
:100BA000070EE66E1CEC26F0456E060EE15E455023
:100BB0000501880E1B6F130E1C6F0501010E196FC6
:100BC00001D000D005011A51010A10E0010A01E02C
:100BD00015D00501190509E181860501100E1D6F6B
:100BE000270E1E6F0501010E1A6F09D005011D5158
:100BF0001E1103E1819605011A6B01D000D021502E
:100C0000000809E235EC0DF0202A030E205C01E11A
:100C1000206A2106F4D72650000809E267EC0DF09F
:100C2000252A030E255C01E1256A2606F4D7200E4D
:100C30000601E76EA819E8AE02D0E73402D0E7500B
:100C4000A85D03E36550020B01E0DDD1400EE66EC6
:100C5000400EE66E020EE66EB4EC31F0E552E5525F
:100C6000E552E76E030EE7CFDBFF030EDB50000813
:100C700001E343D1040EDB6A030EDB50F36E040E76
:100C8000DBCFF4FFF350F45C01E337D1040EDB500B
:100C9000EA6A400FE96E020EEA22EFCFDFFF05019C
:100CA000635145E10D0E456EDF50455C05E00A0ECF
:100CB000466EDF50465C3BE10501010E636F0601A5
:100CC000F751EA6A000FE96E030EEA220D0EEF6E8D
:100CD0000601F72B010EDB6A0601F751F36E010ED8
:100CE000DBCFF4FFF350F45C1CE2010EDBCFE9FF35
:100CF000EA6AE9BEEA68000EE926030EEA22EF502E
:100D0000E66E010EDBCFE9FFEA6AE9BEEA681F0E74
:100D1000E926050EEA22E552E750EF6E010EDB2AC6
:100D2000DBD708DA0601F76B0601F86BD4D01B0E8F
:100D3000DF5C0EE105015F510BE10501010E5F6F04
:100D400005011B0E606F0501616B0501626BC3D06D
:100D500005015F050EE15B0EDF5C0BE11B0E05017B
:100D6000605D07E10501615104E105015B0E616F02
:100D7000B2D005015F056FE1410EDF5C6CE11B0E37
:100D80000501605D68E15B0E0501615D64E10501DF
:100D9000606B0501616B0501626B05015F6B010E04
:100DA000DB6A010EDBCFE9FFEA6AE9BEEA68000E02
:100DB000E926030EEA22EF500D081CE0010EDBCFFE
:100DC000E9FFEA6AE9BEEA681F0EE926050EEA2293
:100DD000EF50E66E010EDBCFE9FFEA6AE9BEEA6892
:100DE000000EE926030EEA22E552E750EF6E010EEF
:100DF000DB2AD7D7010EDBCFF7F60601F751EA6AF7
:100E0000000FE96E030EEA22EF6AD70E456E6C0EF4
:100E1000466E476A45C0E6FF46C0E6FF47C0E6FFAC
:100E2000C3EC37F0E552E552E552000EE66E030ED4
:100E3000E66ED40E456E6C0E466E476A45C0E6FF00
:100E400046C0E6FF47C0E6FFC3EC37F0486E050E2C
:100E5000E15E485040D0080EDF5C1FE10601F7510B
:100E600000081BE20601F7070601F751EA6A000FC6
:100E7000E96E030EEA22EF6AD10E456E6C0E466EE5
:100E8000476A45C0E6FF46C0E6FF47C0E6FFC3EC41
:100E900037F0E552E552E5521ED00D0EDF5C1BE047
:100EA0000A0EDF5C18E0200EDF5C15E30501606BC5
:100EB0000501616B0501626B05015F6B0601F7516E
:100EC000EA6A000FE96E030EEA22DFCFEFFF0501A9
:100ED000636B0601F72B0601F751456E466A000E5B
:100EE000451802E1010E461805E128860601F76B58
:100EF0000601F86B040EDB2ABFD6285001E182D030
:100F000028A010D0CB0E456E6C0E466E476A45C0C9
:100F1000E6FF46C0E6FF47C0E6FFC3EC37F0E55208
:100F2000E552E55228A210D0AC0E456E6C0E466E0E
:100F3000476A45C0E6FF46C0E6FF47C0E6FFC3EC90
:100F400037F0E552E552E55228A410D0900E456ED8
:100F50006C0E466E476A45C0E6FF46C0E6FF47C0D6
:100F6000E6FFC3EC37F0E552E552E55228A610D073
:100F7000740E456E6C0E466E476A45C0E6FF46C06D
:100F8000E6FF47C0E6FFC3EC37F0E552E552E55215
:100F900028A810D0550E456E6C0E466E476A45C0A7
:100FA000E6FF46C0E6FF47C0E6FFC3EC37F0E55278
:100FB000E552E55228AA00D028AC10D0340E456E78
:100FC0006C0E466E476A45C0E6FF46C0E6FF47C066
:100FD000E6FFC3EC37F0E552E552E552000E281467
:100FE00010E01B0E456E6C0E466E476A45C0E6FF6C
:100FF00046C0E6FF47C0E6FFC3EC37F0E552E552D6
:10100000E552286A45D8050EE15C02E2E16AE55244
:10101000E16EE552E7CFD9FF1200D9CFE6FFE1CF6D
:10102000D9FFE652F5C6DFFFDF2A400E456EDF50DE
:10103000455C01E1DF6A0601F651DF5C01E128D879
:101040000601F551EA6A000FE96E020EEA22FE0E71
:10105000DBCFEFFF0601F52B400E0601F55D02E147
:101060000601F56B0601F6510601F55D01E12884E4
:10107000FE0EDBCF45F0466A45BE466845C0F3FF2D
:1010800046C0F4FF00D0E552E552E7CFD9FF120089
:10109000D9CFE6FFE1CFD9FFE6520601F5510601AF
:1010A000F65D43E00601905105E0BDEC32F005EC41
:1010B00019F0F8D70601F6510601D880F5551AE265
:1010C0000601F6510601F55DDF6EDFCFE6FF060192
:1010D000F651466A000F456E020E462245C0E6FFF5
:1010E00046C0E6FF1BEC32F0E552E552E552F5C68C
:1010F000F6F619D0400E0601D880F655DF6EDFCF28
:10110000E6FF0601F651466A000F456E020E4622C2
:1011100045C0E6FF46C0E6FF1BEC32F0E552E55263
:10112000E5520601F66BBDEC32F0E552E552E7CF31
:10113000D9FF1200D9CFE6FFE1CFD9FF040EE12697
:10114000DE6ADD6A020EDB6A030EDB6A0601F85115
:10115000EA6A000FE96E030EEA22EF50E66EE66AD5
:101160001CEC39F0E552E552020EF3CFDBFF06012D
:10117000F82B0601F851456E466A000E451802E14B
:10118000010E461802E10601F86B020EDB50DE6E1E
:10119000DD6A0601F851EA6A000FE96E030EEA22E1
:1011A000EF502C083BE00601F851EA6A000FE96EA7
:1011B000030EEA22EF500D0831E00601F851EA6A09
:1011C000000FE96E030EEA22EF50E66EE66A1CECB1
:1011D00039F0E552E552030EF3CFDBFF0601F82BA1
:1011E0000601F851456E466A000E451802E1010EEF
:1011F000461802E10601F86B020EDBCF47F047C04C
:1012000048F0476A030EDB5000014724456E000E8C
:101210004820466E45C0DEFF46C0DDFF000EDBCF36
:1012200039F0010EDBCF3AF04D0E391802E1510EC4
:101230003A1801E1B6D14D0E391802E1520E3A18B2
:1012400001E1ACD1320E391802E1530E3A1801E136
:10125000A2D1450E391802E1530E3A1801E198D196
:10126000430E391802E1510E3A1801E18ED14B0EAE
:10127000391802E1430E3A1801E184D14C0E3918B5
:1012800002E1420E3A1801E17AD1440E391802E126
:101290004E0E3A1801E170D1490E391802E14E0E96
:1012A0003A1801E166D1420E391802E1510E3A189E
:1012B00001E15CD14C0E391802E1510E3A1801E1FE
:1012C00052D14C0E391802E1530E3A1801E148D1BF
:1012D0004E0E391802E1510E3A1801E13ED14E0E80
:1012E000391802E1530E3A1801E134D1430E39188E
:1012F00002E1530E3A1801E12AD14D0E391802E1EC
:10130000450E3A1801E120D1500E391802E1510E74
:101310003A1801E116D1500E391802E1540E3A186C
:1013200001E10CD1500E391802E1530E3A1801E1D7
:1013300002D14D0E391802E1530E3A1801E1F8D0EE
:10134000470E391802E1500E3A1801E1EED0430E73
:10135000391802E1500E3A1801E1E4D0490E39186B
:1013600002E1430E3A1801E1DAD0490E391802E1E0
:10137000520E3A1801E1D0D0490E391802E1530E4D
:101380003A1801E1C6D0530E391802E1430E3A185B
:1013900001E1BCD0530E391802E1520E3A1801E1B6
:1013A000B2D0530E391802E1530E3A1801E1A8D019
:1013B000530E391802E1420E3A1801E19ED0430E55
:1013C000391802E1420E3A1801E194D0430E39185F
:1013D00002E1520E3A1801E18AD04F0E391802E1AB
:1013E000420E3A1801E180D0570E391802E14D0E35
:1013F0003A1801E177D0520E391802E14D0E3A1831
:101400006FE0440E391802E1500E3A1867E04F0EB3
:10141000391802E1500E3A185EE0490E391802E11F
:10142000500E3A1855E0580E391802E1540E3A1889
:101430004CE0540E391801E13A5045E0410E39189C
:1014400001E13A503EE0560E391801E13A5037E0DA
:10145000490E391801E13A5030E04F0E391801E1D8
:101460003A5029E0550E391802E1430E3A1821E0AE
:10147000580E391802E1430E3A1818E0430E391895
:1014800001E13A5011E0520E391801E13A500AE0F8
:10149000580E391802E1520E3A1801E085D0FCECE2
:1014A00010F0C1D0F7D8BFD08FD9BDD0FFEC10F06D
:1014B000BAD0F4D8B8D047DAB6D0D7DAB4D0F6DAA2
:1014C000B2D005DBB0D034D9AED0F9EC10F0ABD04F
:1014D00040EC0FF0A8D009EC10F0A5D0DEDBA3D0D3
:1014E00097DBA1D055DB9FD0BBEC11F09CD002EC78
:1014F00011F099D0B8EC11F096D0BEEC11F093D069
:10150000C1EC11F090D0C4EC11F08DD0C7EC11F00B
:101510008AD0CAEC11F087D0CDEC11F084D0D0EC99
:1015200011F081D0D3EC11F07ED067EC12F07BD0BB
:10153000BEEC25F078D09BEC27F075D05DEC27F061
:1015400072D040EC27F06FD061EC28F06CD0B5EC95
:1015500024F069D005EC29F066D036EC29F063D090
:1015600052EC29F060D065EC29F05DD082EC29F0D6
:101570005AD0E3EC28F057D0F6EC28F054D0A5EC84
:1015800012F051D0ADEC12F04ED0A1EC29F04BD0BE
:1015900012EC2AF048D022EC34F045D0A1EC2AF02D
:1015A00042D0A2EC2AF03FD0030EDB501AE1020E2B
:1015B000DBCFE6FFE66A020EDBCFE6FFE66AF80E57
:1015C000456E6B0E466E476A45C0E6FF46C0E6FFB5
:1015D00047C0E6FFC3EC37F0486E070EE15E4850A7
:1015E00021D0030EDBCFE6FFE66A020EDBCFE6FF7B
:1015F000E66A030EDBCFE6FFE66A020EDBCFE6FF0C
:10160000E66AD00E456E6B0E466E476A45C0E6FF31
:1016100046C0E6FF47C0E6FFC3EC37F0486E0B0E4E
:10162000E15E485000D00601F851EA6A000FE96E09
:10163000030EEA22EF500D080DE028500BE1520E88
:10164000456E466ADF50451803E1DE52DD5046180C
:1016500001E0288EF7C6F8F6040EE15C02E2E16ACA
:10166000E552E16EE552E7CFD9FF12000601FD51C8
:1016700010E0CC0E456E720E466E476A45C0E6FF1E
:1016800046C0E6FF47C0E6FFC3EC37F0E552E5523F
:10169000E55212004DEC04F0E9DF1200D9CFE6FF6D
:1016A000E1CFD9FF030EE126E66AD9CFE6FFDACF14
:1016B000E6FF010EE66EEFEC13F0E552E552E5525F
:1016C000E552E66AD950010FE66E000EDA20E66EAA
:1016D000020EE66EEFEC13F0E552E552E552E552EC
:1016E000285001E01BD0DF0418E1D950010FE96E4A
:1016F000DACFEAFFEE50ED100BE0010E456E466AC0
:10170000010EDB50451803E1020EDB50461804E1E0
:10171000010EDBCFFDF601D0288CA8DF030EE15CC3
:1017200002E2E16AE552E16EE552E7CFD9FF12002D
:10173000D9CFE6FFE1CFD9FF030EE126020EDB6A27
:10174000E66A1B0EE66E000EE66E030EE66EEFEC2A
:1017500013F0E552E552E552E552E66AD950020F20
:10176000E66E000EDA20E66E010EE66EEFEC13F088
:10177000E552E552E552E552285001E01BD0020E39
:10178000DB500CE11B501C1003E11D6A1E6A05D0E2
:1017900076841BC01DF01CC01EF00BD01B501C100B
:1017A00003E1226A236A05D076841BC022F01CC0A4
:1017B00023F05CDF030EE15C02E2E16AE552E16ED8
:1017C000E552E7CFD9FF1200D9CFE6FFE1CFD9FF2D
:1017D0000A0EE126E66AD9CFE6FFDACFE6FF010E70
:1017E000E66EEFEC13F0E552E552E552E552E66A9B
:1017F000D950010FE66E000EDA20E66E010EE66E9D
:10180000EFEC13F0E552E552E552E552E66AD950A5
:10181000020FE66E000EDA20E66E010EE66EEFECC9
:1018200013F0E552E552E552E552E66AD950040F4D
:10183000E66E000EDA20E66E010EE66EEFEC13F0B7
:10184000E552E552E552E552E66AD950050FE66EDB
:10185000000EDA20E66E010EE66EEFEC13F0E552B4
:10186000E552E552E552E66AD950060FE66E000EE3
:10187000DA20E66E010EE66EEFEC13F0E552E5526B
:10188000E552E552E66AD950070FE66E000EDA20FF
:10189000E66E010EE66EEFEC13F0E552E552E5520E
:1018A000E552E66AD950080FE66E000EDA20E66EC1
:1018B000010EE66EEFEC13F0E552E552E552E5520B
:1018C000E66AD950090FE66E000EDA20E66E010EC8
:1018D000E66EEFEC13F0E552E552E552E552E66AAA
:1018E000D950030FE66E000EDA20E66E010EE66EAA
:1018F000EFEC13F0E552E552E552E552285001E0D5
:1019000018D0DF50926E010EDB50936E020EDB504A
:10191000946E040EDB50956E050EDB50966E030E32
:10192000DB500C0805E20C0EF36E030EF3CFDBFF69
:101930009DDE0A0EE15C02E2E16AE552E16EE552EB
:10194000E7CFD9FF1200D9CFE6FFE1CFD9FF020ED2
:10195000E126E66AD9CFE6FFDACFE6FF010EE66EB2
:10196000EFEC13F0E552E552E552E552E76E010E59
:10197000E7CFDBFF285001E06ED0010EDB5002E123
:10198000DF50896E010EE66ED9CFE6FFDACFE6FFB3
:10199000010EE66EEFEC13F0E552E552E552E5522A
:1019A000E76E010EE7CFDBFF285001E054D0010EB7
:1019B000DB5002E1DF508A6E010EE66ED9CFE6FF02
:1019C000DACFE6FF010EE66EEFEC13F0E552E552DA
:1019D000E552E552E76E010EE7CFDBFF285001E04C
:1019E0003AD0010EDB5002E1DF508B6E010EE66E45
:1019F000D9CFE6FFDACFE6FF010EE66EEFEC13F08B
:101A0000E552E552E552E552E76E010EE7CFDBFF06
:101A1000285001E020D0010EDB5002E1DF508C6E37
:101A2000010EE66ED9CFE6FFDACFE6FF010EE66ED5
:101A3000EFEC13F0E552E552E552E552E76E010E88
:101A4000E7CFDBFF285001E006D0010EDB5002E1BA
:101A5000DF508D6E0BDE020EE15C02E2E16AE552C0
:101A6000E16EE552E7CFD9FF12008450E66EE66AD8
:101A70008350E66EE66A8250E66EE66A8150E66E54
:101A8000E66A8050E66EE66AB30E456E6B0E466EF1
:101A9000476A45C0E6FF46C0E6FF47C0E6FFC3EC25
:101AA00037F0486E0D0EE15E48501200D40E456EC0
:101AB000720E466E476A45C0E6FF46C0E6FF47C065
:101AC000E6FFC3EC37F0E552E552E5521200D9CFFC
:101AD000E6FFE1CFD9FFE652DF6AB10E456E6B0E2D
:101AE000466E476A45C0E6FF46C0E6FF47C0E6FFD0
:101AF000C3EC37F0E552E552E552DF6A2750DF5C70
:101B000032E2DFCF45F0466A45BE4668060E460221
:101B1000F3CF46F0060E4502F3CF45F0F4504626CB
:101B2000000E4526010E46222550020D4550F32495
:101B3000E96E4650F420EA6EEECFE6FFEFCFE6FF07
:101B4000AB0E476E6B0E486E496A47C0E6FF48C051
:101B5000E6FF49C0E6FFC3EC37F04A6E050EE15ED2
:101B60004A50DF2ACBD7D10E456E720E466E476AB9
:101B700045C0E6FF46C0E6FF47C0E6FFC3EC37F0CE
:101B8000E552E552E552E552E552E7CFD9FF1200A2
:101B9000D9CFE6FFE1CFD9FF030EE126E66AD9CF20
:101BA000E6FFDACFE6FF030EE66EEFEC13F0E55248
:101BB000E552E552E552E66AD950020FE66E000E94
:101BC000DA20E66E010EE66EEFEC13F0E552E55218
:101BD000E552E552285001E011D0DECF45F0DDCFCF
:101BE00046F0000E455C100E465807E2DECFE9FFD6
:101BF000DDCFEAFF020EDBCFEFFF38DD030EE15C45
:101C000002E2E16AE552E16EE552E7CFD9FF120048
:101C1000D9CFE6FFE1CFD9FF030EE126E66AD9CF9F
:101C2000E6FFDACFE6FF030EE66EEFEC13F0E552C7
:101C3000E552E552E552285001E025D0DECF45F0CF
:101C4000DDCF46F0000E455C100E465807E2DECFB1
:101C5000E9FFDDCFEAFF020EEFCFDBFF020EDBCFA5
:101C6000E6FFE66AA10E456E6B0E466E476A45C0FA
:101C7000E6FF46C0E6FF47C0E6FFC3EC37F0486E1C
:101C8000050EE15E4850030EE15C02E2E16AE552B6
:101C9000E16EE552E7CFD9FF1200D9CFE6FFE1CFE1
:101CA000D9FF030EE126E66AD9CFE6FFDACFE6FFD9
:101CB000050EE66EEFEC13F0E552E552E552E55203
:101CC000E66AD950010FE66E000EDA20E66E010ECC
:101CD000E66EEFEC13F0E552E552E552E552E66AA6
:101CE000D950020FE66E000EDA20E66E010EE66EA7
:101CF000EFEC13F0E552E552E552E552285001E0D1
:101D0000B5D0020EDB50010802E2288CAFD0010EE4
:101D1000DB50070802E2288CA9D0410E456EDF5047
:101D2000455C1CE1020EDB500DE1010EF36E010E6D
:101D3000DB5004E0D890F336E806FCE1F350E81CF1
:101D400092160BD0010EF36E010EDB5004E0D8901A
:101D5000F336E806FCE1F350921286D0420E456E4F
:101D6000DF50455C1CE1020EDB500DE1010EF36E0D
:101D7000010EDB5004E0D890F336E806FCE1F350A6
:101D8000E81C93160BD0010EF36E010EDB5004E03D
:101D9000D890F336E806FCE1F350931265D0430E79
:101DA000456EDF50455C1CE1020EDB500DE1010E7B
:101DB000F36E010EDB5004E0D890F336E806FCE148
:101DC000F350E81C94160BD0010EF36E010EDB509D
:101DD00004E0D890F336E806FCE1F350941244D0C6
:101DE000440E456EDF50455C1CE1020EDB500DE1F8
:101DF000010EF36E010EDB5004E0D890F336E806D6
:101E0000FCE1F350E81C95160BD0010EF36E010EA9
:101E1000DB5004E0D890F336E806FCE1F35095126D
:101E200023D0450E456EDF50455C1CE1020EDB50B1
:101E30000DE1010EF36E010EDB5004E0D890F33695
:101E4000E806FCE1F350E81C96160BD0010EF36E89
:101E5000010EDB5004E0D890F336E806FCE1F350C5
:101E6000961202D0288C02D036EC0BF0030EE15C07
:101E700002E2E16AE552E16EE552E7CFD9FF1200D6
:101E8000D9CFE6FFE1CFD9FF030EE126020EDB6AD0
:101E9000E66AD9CFE6FFDACFE6FF050EE66EEFEC95
:101EA00013F0E552E552E552E552E66AD950010FCA
:101EB000E66E000EDA20E66E010EE66EEFEC13F031
:101EC000E552E552E552E552285001E098D0010E66
:101ED000DB50070802E2288C92D0410E456EDF509D
:101EE000455C12E1010EDB28456E010E455204E00F
:101EF000E846FE0B4506FCE1E8407F0B8014E76EE8
:101F0000020EE7CFDBFF5ED0420E456EDF50455C30
:101F100012E1010EDB28456E010E455204E0E84651
:101F2000FE0B4506FCE1E8407F0B8114E76E020ED4
:101F3000E7CFDBFF47D0430E456EDF50455C12E133
:101F4000010EDB28456E010E455204E0E846FE0B0B
:101F50004506FCE1E8407F0B8214E76E020EE7CFF6
:101F6000DBFF30D0440E456EDF50455C12E1010EC0
:101F7000DB28456E010E455204E0E846FE0B45069F
:101F8000FCE1E8407F0B8314E76E020EE7CFDBFF36
:101F900019D0450E456EDF50455C12E1010EDB287D
:101FA000456E010E455204E0E846FE0B4506FCE195
:101FB000E8407F0B8414E76E020EE7CFDBFF02D010
:101FC000288C1DD0020EDB5005E0010EF36E020ED0
:101FD000F3CFDBFF020EDBCFE6FFE66A980E456E1D
:101FE0006B0E466E476A45C0E6FF46C0E6FF47C037
:101FF000E6FFC3EC37F0486E050EE15E4850030E75
:10200000E15C02E2E16AE552E16EE552E7CFD9FF19
:102010001200D9CFE6FFE1CFD9FF030EE126E66A31
:10202000D9CFE6FFDACFE6FF050EE66ED8DBE55244
:10203000E552E552E552E66AD950010FE66E000E10
:10204000DA20E66E010EE66ECADBE552E552E55295
:10205000E552E66AD950020FE66E000EDA20E66E0F
:10206000010EE66EBCDBE552E552E552E552285022
:1020700001E0B5D0020EDB50010802E2288CAFD09F
:10208000010EDB50070802E2288CA9D0410E456EF4
:10209000DF50455C1CE1020EDB500DE1010EF36EDA
:1020A000010EDB5004E0D890F336E806FCE1F35073
:1020B000E81C89160BD0010EF36E010EDB5004E014
:1020C000D890F336E806FCE1F350891286D0420E30
:1020D000456EDF50455C1CE1020EDB500DE1010E48
:1020E000F36E010EDB5004E0D890F336E806FCE115
:1020F000F350E81C8A160BD0010EF36E010EDB5074
:1021000004E0D890F336E806FCE1F3508A1265D07B
:10211000430E456EDF50455C1CE1020EDB500DE1C5
:10212000010EF36E010EDB5004E0D890F336E806A2
:10213000FCE1F350E81C8B160BD0010EF36E010E80
:10214000DB5004E0D890F336E806FCE1F3508B1244
:1021500044D0440E456EDF50455C1CE1020EDB505E
:102160000DE1010EF36E010EDB5004E0D890F33662
:10217000E806FCE1F350E81C8C160BD0010EF36E60
:10218000010EDB5004E0D890F336E806FCE1F35092
:102190008C1223D0450E456EDF50455C1CE1020ECB
:1021A000DB500DE1010EF36E010EDB5004E0D89020
:1021B000F336E806FCE1F350E81C8D160BD0010E57
:1021C000F36E010EDB5004E0D890F336E806FCE134
:1021D000F3508D1202D0288C02D036EC0BF0030E97
:1021E000E15C02E2E16AE552E16EE552E7CFD9FF38
:1021F000120036EC0BF0120036EC0BF0120036EC4D
:102200000BF01200D9CFE6FFE1CFD9FF040EE12693
:10221000E66AD9CFE6FFDACFE6FF050EE66EDFDA33
:10222000E552E552E552E552E66AD950010FE66EF5
:10223000000EDA20E66E010EE66ED1DAE552E552C6
:10224000E552E552E66AD950020FE66E000EDA203A
:10225000E66E030EE66EC3DAE552E552E552E5524C
:10226000285001E07BD0D950020FE96EDACFEAFFA7
:10227000720ED880EE542E0EED5402E2288C6ED0F1
:10228000D950020FE96EDACFEAFFEE50ED101FE0F1
:10229000486849684A6A2D0EE76E020EDBCF4BF0A4
:1022A000030EDBCF4CF0E7504B26000E4C224D6A5C
:1022B0004B50485C456E4C504958466E4D504A58FC
:1022C000476E020E45C0DBFF030E46C0DBFF010E6A
:1022D000DB50070802E2288C41D0410E456EDF50EA
:1022E000455C02E1DF6A12D0420E456EDF50455C6C
:1022F00003E1080EDF6E0AD0430E456EDF50455CE9
:1023000003E1100EDF6E02D0288C28D0010EDB50C6
:10231000DF24E96EEA6AD890E936EA36690EE926E2
:10232000010EEA22020EDBCFEEFF030EDBCFEDFF44
:10233000010EDB50DF24EA6A510FE96E010EEA223A
:10234000EF040AE1010EDB50DF24EA6A510FE96E67
:10235000010EEA22020EEF6E36EC0BF0040EE15C89
:1023600002E2E16AE552E16EE552E7CFD9FF1200E1
:1023700036EC0BF0120036EC0BF0120036EC0BF0E2
:10238000120036EC0BF0120036EC0BF0120036ECBB
:102390000BF0120036EC0BF0120036EC0BF01200D2
:1023A00036EC0BF01200D9CFE6FFE1CFD9FF070ED4
:1023B000E126E66AD9CFE6FFDACFE6FF030EE66E46
:1023C0000EDAE552E552E552E552E66AD950020FBF
:1023D000E66E000EDA20E66E030EE66E00DAE552D7
:1023E000E552E552E552285001E067D0DECF01F515
:1023F000DDCF02F5020EDBCF09F5030EDBCF0AF5C8
:10240000040EDB6A030EF36E040EDBCFF4FFF35011
:10241000F45C51E2010EE66ED9CFE6FFDACFE6FFBB
:10242000030EE66EDCD9E552E552E552E552E76E61
:10243000050EE7CFDBFF010EE66ED950020FE66E08
:10244000000EDA20E66E030EE66EC9D9E552E552BB
:10245000E552E552E76E060EE7CFDBFF285001E0BC
:102460002CD0050EDB5003E1060EDB5001E023D03B
:10247000040EDB28E96EEA6AD890E936EA36010EE6
:10248000E926050EEA22DECFEEFFDDCFEDFF040EDA
:10249000DB28E96EEA6AD890E936EA36090EE926C1
:1024A000050EEA22020EDBCFEEFF030EDBCFEDFFBF
:1024B000040EDB2AA7D736EC0BF0070EE15C02E234
:1024C000E16AE552E16EE552E7CFD9FF1200D9CFBC
:1024D000E6FFE1CFD9FFE652E66AD9CFE6FFDACFD1
:1024E000E6FF010EE66E7BD9E552E552E552E55274
:1024F000285001E00DD0DF5007E0F00E9314936EEA
:102500000501010E006F02D00501006B36EC0BF0E7
:10251000E552E552E7CFD9FF1200D9CFE6FFE1CF70
:10252000D9FFE652DF6AFF0EDF5C0AE2E868E85096
:1025300005E0E80600D000D000D0F9D7DF2AF3D7B5
:10254000E552E552E7CFD9FF1200F29EF29C659268
:10255000656AE3DF0FEF00F01200D9CFE6FFE1CFAD
:10256000D9FF100EE126E66AD950010FE66E000E83
:10257000DA20E66EE66A33D9E552E552E552E552D5
:10258000E66AD9CFE6FFDACFE6FF010EE66E27D97D
:10259000E552E552E552E552E66AD950040FE66E7F
:1025A000000EDA20E66E020EE66E19D9E552E5520B
:1025B000E552E552E66AD950020FE66E000EDA20C7
:1025C000E66E030EE66E0BD9E552E552E552E55292
:1025D000E66AD9500A0FE66E000EDA20E66E060EA5
:1025E000E66EFDD8E552E552E552E552E66AD9506D
:1025F000060FE66E000EDA20E66E070EE66EEFD8E6
:10260000E552E552E552E552E66AD9500E0FE66E04
:10261000000EDA20E66E040EE66EE1D8E552E552D1
:10262000E552E552E66AD9500F0FE66E000EDA2049
:10263000E66E050EE66ED3D8E552E552E552E55258
:10264000010EDBCF45F0466A45BE466845C0E6FF51
:1026500046C0E6FF8C0E476E6B0E486E496A47C057
:10266000E6FF48C0E6FF49C0E6FFC3EC37F04A6E1C
:10267000050EE15E4A50DFCFE6FFE66A800E456E4A
:102680006B0E466E476A45C0E6FF46C0E6FF47C090
:10269000E6FFC3EC37F0486E050EE15E4850040ECD
:1026A000DBCFE6FF050EDBCFE6FF740E456E6B0E4B
:1026B000466E476A45C0E6FF46C0E6FF47C0E6FFF4
:1026C000C3EC37F0486E050EE15E4850020EDBCFDA
:1026D000E6FF030EDBCFE6FF680E456E6B0E466E1F
:1026E000476A45C0E6FF46C0E6FF47C0E6FFC3ECC9
:1026F00037F0486E050EE15E4850D9500A0FE96E7A
:10270000DACFEAFFEECFE6FFEECFE6FFEECFE6FF51
:10271000EFCFE6FF5B0E456E6B0E466E476A45C017
:10272000E6FF46C0E6FF47C0E6FFC3EC37F0486E61
:10273000070EE15E4850D950060FE96EDACFEAFF86
:10274000EECFE6FFEECFE6FFEECFE6FFEFCFE6FF00
:102750004E0E456E6B0E466E476A45C0E6FF46C09C
:10276000E6FF47C0E6FFC3EC37F0486E070EE15EB8
:1027700048500E0EDBCFE6FFE66A420E456E6B0E4A
:10278000466E476A45C0E6FF46C0E6FF47C0E6FF23
:10279000C3EC37F0486E050EE15E48500F0EDBCFFC
:1027A000E6FFE66A360E456E6B0E466E476A45C01A
:1027B000E6FF46C0E6FF47C0E6FFC3EC37F0486ED1
:1027C000050EE15E485036EC0BF0100EE15C02E2C3
:1027D000E16AE552E16EE552E7CFD9FF1200D9CFA9
:1027E000E6FFE1CFD9FF090EE126080EDB6A0D0EE8
:1027F000456E0601F851EA6A000FE96E030EEA22FF
:10280000EF50455C06E1FB0EDB5001E12888030E2A
:1028100037D20601F851EA6A000FE96E030EEA2288
:10282000EF502C0821E0FB0EDB501CE10601F851B3
:10283000EA6A000FE96E030EEA22EF50E66EE66ADE
:102840000F0E456E6B0E466E476A45C0E6FF46C0EA
:10285000E6FF47C0E6FFC3EC37F0486E050EE15EC9
:102860004850288A020E0CD20601F82B0601F851B6
:10287000456E466A000E451802E1010E461802E157
:102880000601F86B0D0E456E0601F851EA6A000F5D
:10289000E96E030EEA22EF50455C06E1FB0EDB50C9
:1028A00001E12888030EECD12D0E456E0601F8518A
:1028B000EA6A000FE96E030EEA22EF50455C32E14E
:1028C000040E466EFE0EDB50465C2CE0050E476E95
:1028D000FE0EDB50475C26E0FE0EDB040CE0030E30
:1028E000456EFE0EDB50455C06E0070E466EFE0EA2
:1028F000DB50465C04E1288C010EC2D113D0010EDE
:10290000F36E080EF3CFDBFF0601F82B0601F8513A
:10291000456E466A000E451802E1010E461802E1B6
:102920000601F86B040E456EFE0EDB50455C11E0AF
:10293000050E466EFE0EDB50465C0BE00A0EE66EA0
:10294000D9CFE6FFDACFE6FFA7D9E552E552E55247
:1029500045D00601F851EA6A000FE96E030EEA223B
:10296000EFCF45F0000E45C0DBFF010EDB6A020E23
:10297000DB6A030EDB6A050E456EFE0EDB50455C1E
:102980001FE1000EDBCFE6FF010EDBCFE6FF1CEC04
:1029900039F0E552E552F3CF45F0F4CF46F0476AFF
:1029A000486A46AE02D04768486845C0DFFF010E5E
:1029B00046C0DBFF020E47C0DBFF030E48C0DBFF53
:1029C0000601F82B0601F851456E466A000E4518BF
:1029D00002E1010E461802E10601F86B080EDB5019
:1029E0006EE0FE0EDB500EE1D9CFE9FFDACFEAFF51
:1029F000D880800EEE54000EEE54000EEE54000E01
:102A0000EE5428E3020E456EFE0EDB50455C0EE1EF
:102A1000D9CFE9FFDACFEAFFD880000EEE54800E5E
:102A2000EE54000EEE54000EEE5414E3060E466E05
:102A3000FE0EDB50465C11E1D9CFE9FFDACFEAFFA9
:102A4000D880000EEE54000EEE54000EEE54800EB0
:102A5000EE5403E2288C010E13D1D9CFE9FFDACF6F
:102A6000EAFF040EEECFDBFF050EEECFDBFF060E16
:102A7000EECFDBFF070EEECFDBFF080EDB501EE0D4
:102A8000040EDBCF37F0050EDBCF38F0060EDBCFC0
:102A900039F0070EDBCF3AF03C683D683E683F688E
:102AA000E4EC38F0040E33C0DBFF050E34C0DBFF6E
:102AB000060E35C0DBFF070E36C0DBFF77D0FE0EFB
:102AC000DB500EE1D9CFE9FFDACFEAFFD8807F0EE5
:102AD000EE54000EEE54000EEE54000EEE544DE394
:102AE000FE0EDB040EE1D9CFE9FFDACFEAFFD88092
:102AF000FF0EEE54000EEE54000EEE54000EEE5497
:102B00003CE3020E456EFE0EDB50455C0EE1D9CF74
:102B1000E9FFDACFEAFFD880FF0EEE547F0EEE54C5
:102B2000000EEE54000EEE5428E3030E466EFE0E29
:102B3000DB50465C0EE1D9CFE9FFDACFEAFFD8805F
:102B4000FF0EEE54FF0EEE54000EEE54000EEE5447
:102B500014E3060E476EFE0EDB50475C11E1D9CF41
:102B6000E9FFDACFEAFFD880FF0EEE54FF0EEE54F5
:102B7000FF0EEE547F0EEE5403E2288C010E80D03F
:102B8000070E456EFE0EDB50455C10E0D9CFE9FF25
:102B9000DACFEAFF040EEECFDBFF050EEECFDBFF50
:102BA000060EEECFDBFF070EEECFDBFFFE0EDB5097
:102BB000070A50E0010A3BE0050A2CE0010A1DE08B
:102BC000030A11E0050A0FE0010A0DE0050A01E021
:102BD00053D0FC0EDBCFE9FFFD0EDBCFEAFF040E86
:102BE000DBCFEFFF4BD0FC0EDBCFE9FFFD0EDBCFE1
:102BF000EAFF040EDBCFEFFF41D0FC0EDBCFE9FF95
:102C0000FD0EDBCFEAFF040EDBCFEEFF050EDBCFC0
:102C1000EDFF34D0FC0EDBCFE9FFFD0EDBCFEAFF8A
:102C2000040EDBCFEEFF050EDBCFEDFF27D0FC0E51
:102C3000DBCFE9FFFD0EDBCFEAFF040EDBCFEEFFBB
:102C4000050EDBCFEEFF060EDBCFEEFF070EDBCF70
:102C5000EEFF14D0FC0EDBCFE9FFFD0EDBCFEAFF69
:102C6000DFCFEEFF010EDBCFEEFF020EDBCFEEFF7C
:102C7000030EDBCFEEFF02D0040E02D0000E00D018
:102C8000456E090EE15C02E2E16AE552E16E4550F3
:102C9000E552E7CFD9FF1200D9CFE6FFE1CFD9FF48
:102CA000020EE126FD0EDBCFE9FFFE0EDBCFEAFFD1
:102CB000EE6AEE6AEE6AEE6A010EDB6AFC0EDB502B
:102CC000F36E010EDBCFF4FFF350F45C64E2060117
:102CD000F851EA6A000FE96E030EEA22EFCFDFFF38
:102CE000300EDF5C53E3DF50390850E3FD0EDBCFDD
:102CF000E9FFFE0EDBCFEAFFEECF45F0EECF46F068
:102D0000EECF47F0EFCF48F00A0E3C6E3D6A3E6AC8
:102D10003F6A45C037F046C038F047C039F048C078
:102D20003AF0E4EC38F033C045F034C046F035C03A
:102D300047F036C048F0300EDF5C496E4A6A4B6A95
:102D40004C6A495045264A5046224B5047224C5027
:102D50004822FD0EDBCFE9FFFE0EDBCFEAFF45C0C8
:102D6000EEFF46C0EEFF47C0EEFF48C0EEFF060193
:102D7000F82B0601F851456E466A000E451802E12F
:102D8000010E461802E10601F86B02D0000E05D0D4
:102D9000010EDB2A93D7010E00D0456E020EE15CD6
:102DA00002E2E16AE552E16E4550E552E7CFD9FF14
:102DB00012002150E66EE66A030E456E6B0E466EFB
:102DC000476A45C0E6FF46C0E6FF47C0E6FFC3ECE2
:102DD00037F0486E050EE15E485012000601A8511A
:102DE00008E0010E456E6550020B01E0010E455CE6
:102DF00022E105016707000E685B050169510EE1DC
:102E000005016751681109E18C860501A00E676F05
:102E10000F0E686F0501010E696F0CD00501675137
:102E2000681108E18C960501A00E676F0F0E686FA0
:102E30000501696B79D00601A8050CE0020E0601B8
:102E4000A85D08E0040E0601A85D04E0100E06016E
:102E5000A85D22E105016707000E685B0501695165
:102E60000EE105016751681109E18C860501200E0C
:102E7000676F4E0E686F0501010E696F0CD005017A
:102E80006751681108E18C960501200E676F4E0EA0
:102E9000686F0501696B48D0200E0601A85D44E10A
:102EA00005016707000E685B050169510EE1050128
:102EB0006751681109E18C860501100E676F270EB6
:102EC000686F0501010E696F2FD0050169050EE1DC
:102ED00005016751681109E18C960501100E676FB5
:102EE000270E686F0501020E696F1ED0020E0501E4
:102EF000695D0EE105016751681109E18C860501E4
:102F0000A00E676F860E686F0501030E696F0CD007
:102F100005016751681108E18C960501100E676F75
:102F2000270E686F0501696B1200D9CFE6FFE1CF6C
:102F3000D9FFFE0EDBCF45F0190EE76E4518E8AE5F
:102F400002D0453403D0E750D880455401E253D035
:102F5000FD0EDB5028E0FE0EDBCFE9FFEA6AE9BE9A
:102F6000EA68CE0EE926050EEA22EF50466E010E03
:102F7000465204E0E846FE0B4606FCE1456EFE0EB6
:102F8000DBCFE9FFEA6AE9BEEA68D890E936EA36BB
:102F90009C0EE926050EEA22EE50EFCFEAFFE96E1D
:102FA0004550EF1228D0FE0EDBCFE9FFEA6AE9BEFA
:102FB000EA68CE0EE926050EEA22EF50466E010EB3
:102FC000465204E0E846FE0B4606FCE1E81C456E6E
:102FD000FE0EDBCFE9FFEA6AE9BEEA68D890E9367F
:102FE000EA369C0EE926050EEA22EE50EFCFEAFF04
:102FF000E96E4550EF16E552E7CFD9FF1200D9CF61
:10300000E6FFE1CFD9FFFE0EDBCF45F0190EE76EEC
:103010004518E8AE02D0453403D0E750D880455477
:1030200001E253D0FD0EDB5029E1FE0EDBCFE9FFBC
:10303000EA6AE9BEEA68CE0EE926050EEA22EF50FA
:10304000466E010E465204E0E846FE0B4606FCE1E1
:10305000E81C456EFE0EDBCFE9FFEA6AE9BEEA68CE
:10306000D890E936EA366A0EE926050EEA22EE50D5
:10307000EFCFEAFFE96E4550EF1627D0FE0EDBCF0B
:10308000E9FFEA6AE9BEEA68CE0EE926050EEA2201
:10309000EF50466E010E465204E0E846FE0B46062F
:1030A000FCE1456EFE0EDBCFE9FFEA6AE9BEEA68A5
:1030B000D890E936EA366A0EE926050EEA22EE5085
:1030C000EFCFEAFFE96E4550EF12E552E7CFD9FFA7
:0230D0001200EC
:0E30D200D9CFE6FFE1CFD9FFE652A098636A9E
:1030E000626A0F01266B020EE66EE66AE66A270E3A
:1030F000E66E0F0EE66E76EC37F0456E050EE15E7D
:1031000045500F01160E396F0F019F0E376F0F01DB
:103110007B0E366FDF6ADF50456E466A0C0E455CEB
:10312000000E465810E2DF50040DF3CFE9FFF4CF54
:10313000EAFF000EE926040EEA22EE6AEE6AEE6A63
:10314000EE6ADF2AE8D7658C0F01386B6598659CBD
:1031500062A609D062960601BF6B0601C46B060128
:10316000C56BC66BF5D70601010ED86F0601010EBF
:10317000D96F0601DA6B0601DB6B0601CC6BDF6AE7
:10318000030EDF5C26E2EA6ADF34FE0BEA36E96E04
:10319000B50EE926060EEA22EE6AED6AEA6ADF3427
:1031A000FE0BEA36E96EAF0EE926060EEA22EE6A5B
:1031B000ED6ADF50EA6AD00FE96E060EEA22EF6A86
:1031C000DF50EA6AD30FE96E060EEA22EF6ADF2AC1
:1031D000D7D70601080EB56F040EB66F0F01160E95
:1031E000266F0401300E026F040E036F0401400EBF
:1031F000016F0401840E006F0601A96B0601A86B24
:10320000E552E552E7CFD9FF1200D9CFE6FFE1CF73
:10321000D9FFE65282BE07D0656A0F01366B060100
:10322000A86BA198DCD00601A85113E1656A0F01D3
:10323000366B0F01160E396F0F019F0E376F0F019E
:103240007B0E366F65B602D06586FCD70601010E8F
:10325000A86F0601A8050CE165BA0AD0626A0F01E1
:10326000366B0F0136810F0136890601020EA86FF9
:103270006250040B08E00F010F013651040B03E00C
:10328000629470EC1FF065A202D0A198A8D06250A1
:10329000010B0AE00F010F013651010B05E019DFA8
:1032A0000601040EA86F62906250100B08E00F0137
:1032B0000F013651100B03E059EC1FF0629862AC1D
:1032C0001CD00F0136AD0FD0010EE66EE66A000E7F
:1032D000E66EE66A730EE66EE66AD7EC36F0456E89
:1032E000060EE15E4550629C0601D65102E00601E1
:1032F000D6070601D65101E1F9D96250200B07E04B
:103300000F010F013651200B02E03EEC1FF062501E
:10331000020B15E00F010F013651020B10E0010EF8
:10332000E66EE66A000EE66EE66AE6687F0EE66E18
:10333000D7EC36F0456E060EE15E4550636A040E2A
:103340000601E76EA819E8AE02D0E73402D0E750D4
:10335000A85D02E2A19843D00F0136A73FD0DF6AF3
:10336000040EDF5C3BE262A636D064CFCDF60601E8
:10337000CD51780BE842E842E8420601CE6F6296F2
:103380000601CDB509D00601CE51EA6AD30FE96E28
:10339000060EEA22EF7008D00601CE51EA6AD00F7D
:1033A000E96E060EEA22EF700601CE5103E189ECC8
:1033B0001FF010D0000EE66EE66ACD0EE66E060E29
:1033C000E66E720EE66EE66AD7EC36F0456E060ED5
:1033D000E15E455001D002D0DF2AC2D7A198E55264
:1033E000E552E7CFD9FF1200D9CFE6FFE1CFD9FFF1
:1033F000020EE126FD0EDBA407D0E66AFE0EDBCF4F
:10340000E6FF0FDAE552E552FD0EDBA208D0010E11
:10341000E66EFE0EDBCFE6FF04DAE552E552FE0E65
:10342000DB50466A260F456E0F0E462245C0DEFF72
:1034300046C0DDFFDECFE9FFDDCFEAFFFD0EDBCFCB
:10344000EFFF020EE15C02E2E16AE552E16EE55255
:10345000E7CFD9FF1200D9CFE6FFE1CFD9FF020EA7
:10346000E126FD0EDB500FE0FE0EEA6ADB34FE0BB8
:10347000EA36E96EB50EE926060EEA22EECFDEFF49
:10348000EDCFDDFF0ED0FE0EEA6ADB34FE0BEA362E
:10349000E96EAF0EE926060EEA22EECFDEFFEDCF93
:1034A000DDFFD9CFE9FFDACFEAFFEE50ED1003E1FF
:1034B000F36AF46A49D0DECFE9FFDDCFEAFF020EFE
:1034C000E926000EEA22FB0EDBCFEEFFFC0EDBCF7F
:1034D000EDFFDECFE9FFDDCFEAFFEE52FA0EDBCFE4
:1034E000EFFF400E456EDECFE9FFDDCFEAFF45502E
:1034F000EF16880E456EDECFE9FFDDCFEAFF4550BF
:10350000EF12FD0EDB500CE0FE0EEA6ADB34FE0B20
:10351000EA36E96EB50EE926060EEA22EF740BD004
:10352000FE0EEA6ADB34FE0BEA36E96EAF0EE926E0
:10353000060EEA22EF74DECF45F0DDCF46F045C03F
:10354000F3FF46C0F4FF00D0020EE15C02E2E16A44
:10355000E552E16EE552E7CFD9FF1200D9CFE6FF81
:10356000E1CFD9FF020EE126FE0EDB5020E1ADC611
:10357000E9FFAEC6EAFFEE52400EEF6EADC6E9FFC0
:10358000AEC6EAFF020EE926000EEA22300EEE6E0B
:10359000040EED6EADC6E9FFAEC6EAFF8C0EEF6E0F
:1035A000B5C6E9FFB6C6EAFF840EEF6E3DD0FD0E4C
:1035B000DB50E824476EFE0EDB50040DF350472429
:1035C000040DF3CF45F0F4CF46F0000E4526040E6F
:1035D000462245C0DEFF46C0DDFF840E456EDECFCD
:1035E000E9FFDDCFEAFF4550EF12FD0EDB50E82486
:1035F000476EFE0EDB50040DF3504724010F040DFF
:10360000F3CF45F0F4CF46F0000E4526040E4622D7
:1036100045C0DEFF46C0DDFF840E456EDECFE9FF0C
:10362000DDCFEAFF4550EF12020EE15C02E2E16AF3
:10363000E552E16EE552E7CFD9FF1200D9CFE6FFA0
:10364000E1CFD9FF65A84ED0FE0EEA6ADB34FE0B4F
:10365000EA36E96EB50EE926060EEA22EE50EFCF05
:10366000EAFFE96E400EEE16EE6AEE6AEE6AFE0EB4
:10367000EA6ADB34FE0BEA36E96EB50EE926060E81
:10368000EA22EE50EFCFEAFFE96EEE7CFE0EEA6A28
:10369000DB34FE0BEA36E96EB50EE926060EEA22A9
:1036A000EF74400E456EFE0EEA6ADB34FE0BEA361E
:1036B000E96EB50EE926060EEA22EE50EFCFEAFFDC
:1036C000E96E4550EF16FE0EEA6ADB34FE0BEA3671
:1036D000E96EB50EE926060EEA22EE50EFCFEAFFBC
:1036E000E96EEF7CE552E7CFD9FF12000601D85111
:1036F00054E10601010ED86F0601D9514EE10601D1
:10370000010ED96F020E0601BC5D0DE1B5C6E9FFE1
:10371000B6C6EAFFEE52EF6AB5C6E9FFB6C6EAFFE3
:10372000C80EEF6E3AD00601BC0537E10601CF6B3B
:10373000ABC6E9FFACC6EAFFEE52400EEF6EABC679
:10374000E9FFACC6EAFF020EE926000EEA22300EBF
:10375000EE6E040EED6EABC6E9FFACC6EAFF840E5A
:10376000EF6E0601010ECF6FADC6E9FFAEC6EAFFF0
:10377000EE52400EEF6EADC6E9FFAEC6EAFF020E96
:10378000E926000EEA22300EEE6E040EED6EADC696
:10379000E9FFAEC6EAFF800EEF6E12000601DA6B9B
:1037A0000601DB6B020E0601BC5D1AE1ADC6E9FF46
:1037B000AEC6EAFFEE52400EEF6EADC6E9FFAEC6F2
:1037C000EAFF020EE926000EEA22380EEE6E040E23
:1037D000ED6EADC6E9FFAEC6EAFFC80EEF6E20D0B3
:1037E0000601C0510401365D0601C151040137597B
:1037F00004E236C4C0F637C4C1F6DBD8B5C6E9FF6B
:10380000B6C6EAFF020EE926000EEA22380EEE6E78
:10381000040EED6EB5C6E9FFB6C6EAFFC80EEF6E40
:103820001200D9CFE6FFE1CFD9FF020EE126000E4C
:10383000DE6E040EDD6EFD0EDB50E824476EFE0EDC
:10384000DB50040DF3504724040DF3CF45F0F4CFC3
:1038500046F0D9CFE9FFDACFEAFF4550EE264650D1
:10386000ED22DECFE9FFDDCFEAFFEF9EFD0EDB505C
:103870000FE1FE0EEA6ADB34FE0BEA36E96EAF0EAC
:10388000E926060EEA22DECFEEFFDDCFEDFF0ED0F9
:10389000FE0EEA6ADB34FE0BEA36E96EB50EE92667
:1038A000060EEA22DECFEEFFDDCFEDFFDECFE9FF31
:1038B000DDCFEAFFEF9CDECFE9FFDDCFEAFF040EAC
:1038C000E926000EEA22EF8C020EE15C02E2E16AD8
:1038D000E552E16EE552E7CFD9FF12006598060187
:1038E000BFBF2FD00601C4AF0CD00601020EBC6FC3
:1038F0000601DB5101E152DF0601D96B0601D86BED
:103900001FD0ADC6E9FFAEC6EAFFEE52400EEF6E25
:10391000ADC6E9FFAEC6EAFF020EE926000EEA22B6
:10392000300EEE6E040EED6EADC6E9FFAEC6EAFFD8
:103930008C0EEF6EB5C6E9FFB6C6EAFF840EEF6ED9
:1039400037D0040130AF10D00601010EBC6F060164
:10395000DA5101E123DF0601D96B0601D86B0601BC
:10396000D75101E1C3DE24D00601020EBC6FADC603
:10397000E9FFAEC6EAFFEE52400EEF6EADC6E9FFBC
:10398000AEC6EAFF020EE926000EEA22300EEE6E07
:10399000040EED6EADC6E9FFAEC6EAFF840EEF6E13
:1039A0000601D96B0601D86B0601D75101E19EDEF5
:1039B0001200D9CFE6FFE1CFD9FFE652400EDF6E0D
:1039C0000601400EC05D000EC1590FE2C0C6DFFF08
:1039D0000601BB5104E10601010EBB6F06D00601D2
:1039E000BB0503E10601020EBB6FDF50456E466A60
:1039F00045500601C05D0601C06F46500601C15921
:103A00000601C16FB5C6E9FFB6C6EAFFEE52DFCFC9
:103A1000EFFF0601380EC96F040ECA6F0601BFB171
:103A20001BD0DF5018E00601BDC6F6FFBEC6F7FF8B
:103A3000BD2B000EBE230800F550E66E0601C9C678
:103A4000E9FFCAC6EAFFC92B000ECA23E552E750B8
:103A5000EF6EDF06E6D719D0DF5017E00601BDC6CE
:103A6000E9FFBEC6EAFFBD2B000EBE23EF50E66E97
:103A70000601C9C6E9FFCAC6EAFFC92B000ECA2360
:103A8000E552E750EF6EDF06E7D7E552E552E7CFA4
:103A9000D9FF1200D9CFE6FFE1CFD9FF020EE12610
:103AA000ABC6E9FFACC6EAFFEE52EFCFDFFFDFCFD8
:103AB00045F045500601C55D000EC65902E2C5C677
:103AC000DFFFDF50456E466A45500601C55D0601C1
:103AD000C56F46500601C6590601C66F010EDB6A66
:103AE000DF50F36E010EDBCFF4FFF350F45C17E20E
:103AF000010EDB50EA6A380FE96E040EEA22EF503D
:103B0000E66E0601C2C6E9FFC3C6EAFFC22B000E7D
:103B1000C323E552E750EF6E010EDB2AE1D7060121
:103B2000000ED880C555000EC65528E2ADC6E9FF87
:103B3000AEC6EAFFEE52400EEF6EADC6E9FFAEC66E
:103B4000EAFF020EE926000EEA22380EEE6E040E9F
:103B5000ED6EABC6E9FFACC6EAFFEF50400B07E1E4
:103B6000ADC6E9FFAEC6EAFFC80EEF6E06D0ADC621
:103B7000E9FFAEC6EAFF880EEF6E2AD0ADC6E9FFB8
:103B8000AEC6EAFFEE52400EEF6EADC6E9FFAEC61E
:103B9000EAFF020EE926000EEA22300EEE6E040E57
:103BA000ED6EADC6E9FFAEC6EAFF840EEF6E06010C
:103BB000C751C81107E005D0C8C6FAFF0601C751B2
:103BC000F96EFADF0601C49F0601D75101E18EDDCF
:103BD000020EE15C02E2E16AE552E16EE552E7CFF6
:103BE000D9FF1200D9CFE6FFE1CFD9FFE652060197
:103BF000BF8F020EE66EE66AE66A270EE66E0F0ECD
:103C0000E66E76EC37F0456E050EE15E4550300EFF
:103C1000E66EE66AE66A000EE66E040EE66E76EC86
:103C200037F0456E050EE15E4550658CDF6A030E88
:103C3000DF5C10E2DF50EA6AD00FE96E060EEA227E
:103C4000EF6ADF50EA6AD30FE96E060EEA22EF6AE6
:103C5000DF2AEDD7010EE66EE66AE66AAA0EE66E88
:103C6000060EE66E76EC37F0456E050EE15E4550C9
:103C7000659C0601080EB56F040EB66F0601000EB6
:103C8000AB6F040EAC6FABC6ADF6ACC6AEF632C4CD
:103C9000A9F60601A95104E10601100EA86F13D080
:103CA000010EE66EE66AA90EE66E060EE66E010EDF
:103CB000E66EE66AD7EC36F0456E060EE15E4550DC
:103CC0000601200EA86FE552E552E7CFD9FF12009A
:103CD000800E0401305D61E10601C00EBF6F04017A
:103CE0003351030A35E0010A0DE0030A01E052D026
:103CF0000601B40EBD6F700EBE6F120E0601C06FCE
:103D0000C16B4BD004013251F66EF76AD890F6368B
:103D1000F7363B0EF626710EF7220900F5CFBDF6F9
:103D20000A00F5CFBEF6020E0601F76ABD25F66E53
:103D3000BE51F7220800F5CFC0F6030E0601F76A60
:103D4000BD25F66EBE51F7220800F5CFC1F625D08D
:103D5000030E0401325D1BE204013251F66EF76A74
:103D6000D890F636F7363D0EF626710EF72209008A
:103D7000F5CFBDF60A00F5CFBEF6BDC6F6FFBEC64E
:103D8000F7FF0800F5500601C06FC16B02D00601B5
:103D9000BF6B03D00601BF6B00D01200D9CFE6FF86
:103DA000E1CFD9FF020EE1260401386B0401396B23
:103DB000040130511F0B020A12E0030A0DE0010A50
:103DC00001E045D00601BF8F040138810601CB0513
:103DD00002E1040138833BD00601BF8F38D00601D1
:103DE000BF8F040134BF11D0040134510F0BE96EB1
:103DF000EA6AD890E936EA36AF0EE926060EEA22DC
:103E0000EECFDEFFEDCFDDFF10D0040134510F0BFC
:103E1000E96EEA6AD890E936EA36B50EE926060E6A
:103E2000EA22EECFDEFFEDCFDDFFDECFE9FFDDCF13
:103E3000EAFFEF50800B0AE0DECFE9FFDDCFEAFFBB
:103E4000EF50040B03E00401010E386F00D00601AF
:103E5000BFAF0AD00601380EBD6F040EBE6F06015B
:103E6000BF810601020EC06F020EE15C02E2E16A50
:103E7000E552E16EE552E7CFD9FF12000F0126A10E
:103E800016D0ABC6E9FFACC6EAFFEF5080080DE1E3
:103E9000B5C6E9FFB6C6EAFFEF50840806E1ABC637
:103EA000E9FFACC6EAFF8C0EEF6E0F012691629A15
:103EB00012000F013685629865820601010ECC6FF3
:103EC000000EE66EE66A000EE66EE66A750EE66EB7
:103ED000E66AD7EC36F0456E060EE15E45501200FC
:103EE0000601CC6B000EE66EE66A000EE66EE66A30
:103EF000740EE66EE66AD7EC36F0456E060EE15EAD
:103F0000455065920F01369562A402D06294FCD7A9
:103F10001200D9CFE6FFE1CFD9FFE65206012D0E00
:103F2000D66FFD0E0601CD1558E17E0E0601CD15AA
:103F3000E8407F0B040DF3CFABF6F4CFACF6000EE8
:103F40000601AB27040E0601AC23ABC6ADF6ACC62A
:103F5000AEF60601AD75ABC6E9FFACC6EAFFEF50A1
:103F60003C0BE842E8420D0836E1DF6A080EDF5CF0
:103F700024E2ABC6E9FFACC6EAFF020EE926000E5A
:103F8000EA22EE50EFCFEAFFE96EEF50E66EDF5027
:103F9000EA6A300FE96E040EEA22E552E750EF6E4E
:103FA000ABC6E9FFACC6EAFF020EE926000EEA2224
:103FB000EE2A000EEF22DF2AD9D7ABC6E9FFACC646
:103FC000EAFF020EE926000EEA22300EEE6E040E23
:103FD000ED6E0ED801D047D806D0FD0E0601CD15E6
:103FE000040801E168D8E552E552E7CFD9FF120095
:103FF0000601BB6B0601D76B0601DA6B0601DB6BB2
:104000000601CF6B0601BC6BB5C6E9FFB6C6EAFF79
:10401000EF9E0601B575B5C6E9FFB6C6EAFFEF9E8D
:104020000601B575ADC6E9FFAEC6EAFFEF9E060113
:10403000BF6B0601C06BC16B0601C46B0601C56B8B
:10404000C66B9BD8000EE66EE66A000EE66EE66A68
:10405000030EE66EE66AD7EC36F0456E060EE15EBC
:1040600045503CDC1200020E0601BC5D02E112DD8F
:1040700021D00601BC6B0601CF511AE1ADC6E9FFA4
:10408000AEC6EAFFEE52400EEF6EADC6E9FFAEC619
:10409000EAFF020EE926000EEA22300EEE6E040E52
:1040A000ED6EADC6E9FFAEC6EAFF8C0EEF6E02D034
:1040B0000601CF6B1200D9CFE6FFE1CFD9FFE65260
:1040C000B5C6E9FFB6C6EAFFEF50400B01E0010EAE
:1040D000DF6E0601B575080E0601A85D0CE132C45D
:1040E00038FF0F01385104E00601100EA86F03D00D
:1040F0000601040EA86F0601BC0528E1B5C6E9FF5C
:10410000B6C6EAFF020EE926000EEA22380EEE6E6F
:10411000040EED6E4EDC020E0601BB5D07E1B5C676
:10412000E9FFB6C6EAFF840EEF6E0FD0DF5007E15D
:10413000B5C6E9FFB6C6EAFFC80EEF6E06D0B5C633
:10414000E9FFB6C6EAFF880EEF6E12D00601C4AFD3
:104150000DD00601C751C81107E005D0C8C6FAFF47
:104160000601C751F96EFADF0601C49F0601BC6B58
:10417000E552E552E7CFD9FF120004013051600B40
:10418000E842E842E842E842E842000901E064D03F
:10419000040131510C0A5FE00B0A4DE00C0A3FE0CC
:1041A000010A2AE00B0A26E0020A24E0030A20E0C2
:1041B000080A11E0010A0DE00F0A09E0030A01E014
:1041C0004AD00601BF8F0601080EA86F45D080DDDA
:1041D00043D008DD41D00601A90EBD6F060EBE6FAB
:1041E0000601BF810601010EC06F0601BF8F34D0EA
:1041F000D5DD32D032D830D0040134510601BD6F44
:10420000BE6BAA0E0601BD27060E0601BE230601DF
:10421000BF810601010EC06F0601BF8F1DD00601D0
:10422000BF8F04013451EA6AAA0FE96E060EEA2232
:1042300032C4EFFF11D0000EE66EE66A000EE66EA5
:10424000E66A020EE66EE66AD7EC36F0456E060EBA
:10425000E15E455001D000D01200D9CFE6FFE1CF9A
:10426000D9FF050EE1260401320511E104013051A8
:104270001F0B00090CE10601BF8F030E0401315D25
:1042800004E10601010ECB6F02D00601CB6B0401E5
:10429000325101E031D1040130511F0B020801E01D
:1042A0002BD1040134510F0B000901E125D1040188
:1042B00034510F0B020801E21FD1200E0601A85D48
:1042C00001E01AD10601BF8F040134BF1CD00401E4
:1042D00034510F0BE96EEA6AD890E936EA36AF0E30
:1042E000E926060EEA22EECFDEFFEDCFDDFF040168
:1042F00034510F0BEA6AD30FE96E060EEA22020E62
:10430000EFCFDBFF1BD0040134510F0BE96EEA6ADB
:10431000D890E936EA36B50EE926060EEA22EECF47
:10432000DEFFEDCFDDFF040134510F0BEA6AD00F41
:10433000E96E060EEA22020EEFCFDBFFD950020F24
:10434000E96EDACFEAFFEF50010B03E1000EDB94D8
:1043500001D0DF84040134BF11D0040134510F0BAC
:10436000E96EEA6AD890E936EA36AF0EE926060E1B
:10437000EA22DECFEEFFDDCFEDFF10D00401345195
:104380000F0BE96EEA6AD890E936EA36B50EE926EF
:10439000060EEA22DECFEEFFDDCFEDFF030E0401B5
:1043A000315D26E1DECFE9FFDDCFEAFFEF50800B84
:1043B00016E0040134BF0AD0040134510F0BEA6A3D
:1043C000D30FE96E060EEA22EF8209D004013451C0
:1043D0000F0BEA6AD00FE96E060EEA22EF82840E16
:1043E000456EDECFE9FFDDCFEAFF4550EF1284D006
:1043F000DF74DECFE9FFDDCFEAFFEF50800B1BE07B
:10440000DECFE9FFDDCFEAFFEF9EDECFE9FFDDCFB4
:10441000EAFFEF8C020EE66EE66ADECFE6FFDDCF46
:10442000E6FF050EE66EE66AD7EC36F0456E060E40
:10443000E15E455005D0DECFE9FFDDCFEAFFEF8C2E
:10444000DF74D950020FE96EDACFEAFFEF50020BAA
:1044500007E1DECFE9FFDDCFEAFFEF50800B2FE071
:10446000040134BF0AD0040134510F0BEA6AD30FA0
:10447000E96E060EEA22EF9209D0040134510F0BC7
:10448000EA6AD00FE96E060EEA22EF923B0E456E05
:10449000DECFE9FFDDCFEAFF4550EF16020EE66EF4
:1044A000E66ADECFE6FFDDCFE6FF050EE66EE66AE2
:1044B000D7EC36F0456E060EE15E455008D03B0E57
:1044C000456EDECFE9FFDDCFEAFF4550EF16040170
:1044D00034510F0B466A260F456E0F0E4622030E0F
:1044E00045C0DBFF040E46C0DBFF030EDBCFE9FF58
:1044F000040EDBCFEAFFEF90050EE15C02E2E16A19
:0C450000E552E16EE552E7CFD9FF120052
:04450C00DACFE4FF1F
:10451000E2CFDAFFE9CFE4FFEACFE4FFE652D9CFFA
:10452000E6FFE1CFD9FFE6529EA07CD19E908E0E91
:10453000CE6ECF680950166E176A010E186E0A50BB
:104540000B1003E00A06000E0B5A0A500B1002E093
:10455000186A31D1000401E091D00550061004E141
:104560000750081001E189D00101E8510BE009A2D0
:1045700002D08C8E01D08C9E09A602D08C8A01D0EC
:104580008C9A0AD009A202D08C8E01D08C9E09A6EA
:1045900002D08C8A01D08C9A055006101DE0125072
:1045A0000124126E13500220136E000ED880125494
:1045B000800E135410E212C012F013C013F0000E5C
:1045C000125E800E135A010E1610166E010E176E33
:1045D0000506000E065A186A075008101DE0145010
:1045E0000324146E15500420156E000ED880145448
:1045F000800E155410E214C014F015C015F0000E12
:10460000145E800E155A040E1610166E010E176EEB
:104610000706000E085A186A17502FE00101E851EA
:1046200005E016B08C8C16B48C8804D016B08B8242
:1046300016B48C880000000000000000000000009C
:10464000000000000000000000000000000000006A
:10465000000000000000000000000000000000005A
:10466000000000000000000000000101E85103E02C
:104670008C9C8C9802D08B928C989DD0030E005C01
:1046800001E099D00101F55101E177D00F04DF6E0F
:104690000C500D1037E1DF50EA6A310FE96E0E0E53
:1046A000EA22EF500E01EA6AAC25E96EAD51EA222A
:1046B000EF6AEA6ADF34FE0BEA36E96E790EE92624
:1046C0000E0EEA22EE6AED6AEA6ADF34FE0BEA3683
:1046D000E96E490EE9260E0EEA22EE6AED6ADF5017
:1046E000EA6A310FE96E0E0EEA22EF6AEA6ADF34F7
:1046F000FE0BEA36E96E010EE9260E0EEA22EE6A9C
:10470000ED6A3BD0EA6ADF34FE0BEA36E96E790ED9
:10471000E9260E0EEA2210C0EEFF11C0EDFFEA6A94
:10472000DF34FE0BEA36E96E490EE9260E0EEA2268
:104730000CC0EEFF0DC0EDFFDF50EA6A310FE96EED
:104740000E0EEA220EC0EFFFEA6ADF34FE0BEA36F5
:10475000E96E010EE9260E0EEA22EE50ED100DE193
:10476000EA6ADF34FE0BEA36E96E010EE9260E0E28
:10477000EA220CC0EEFF0DC0EDFF0E01B6510E5C3B
:104780001AE10E01B0510C1802E1B1510D180AE105
:104790000101010EE96F0101E56B0101F45101E036
:1047A0008A9809D00101E96B0101010EE56F010151
:1047B000F45101E08A88185029E0006A1A5026E175
:1047C00099C100F09AC101F09BC102F09CC103F0B5
:1047D0009DC104F09EC105F09FC106F0A0C107F085
:1047E000A1C108F0A2C109F0A3C10AF0A4C10BF055
:1047F000A5C10CF0A6C10DF0A7C10EF0A8C10FF025
:10480000A9C110F0AAC111F0010E1A6E8050800BE0
:1048100006E00101F05106E08150010B03E10101C6
:10482000010EEF6FE552E552E7CFD9FFE552E5CF34
:10483000EAFFE5CFE9FFE5CFDAFF1100D9CFE6FFC8
:10484000E1CFD9FFE652DF6ADFCF45F0020EE76E17
:104850004518E8AE02D0E73402D0E750455C1FE2CD
:10486000DFCFE9FFEA6AE9BEEA68D890E936EA36BE
:10487000010EE926000EEA22010EEE6EED6ADFCF90
:10488000E9FFEA6AE9BEEA68D890E936EA36050E39
:10489000E926000EEA22EE6AED6ADF2AD5D7010E7C
:1048A0001A6ECD92CD9ECD9CCD8ACD98CD96CD94CD
:1048B0008E0ECE6ECF68CD809F809E909D80928020
:1048C0000F01FE0E486F0F01170E496F8D849694ED
:1048D0008D829692898C929C8D8096908B829492F8
:1048E0008C9C959C8C9E959E8C9895988C9A959A6C
:1048F000949E828E00000000000000000000000076
:1049000000000000000000000000000000000000A7
:1049100000000000000000000000948E829E010153
:10492000010EF46F0101010EF56F8A989398010151
:10493000010EE56F0101010EE86F0101010EE96F43
:104940000101EE6B0101EA6BEB6BEC6BED6B0101AE
:10495000EF6B9380F19E0101010EF06F93968196AB
:10496000E552E552E7CFD9FF1200D9CFE6FFE1CFFC
:10497000D9FF030EE126DF6A010EDB6A020EDB6A55
:10498000E66AD9CFE6FFDACFE6FF010EE66EEFEC7E
:1049900013F0E552E552E552E552E66AD950010FAF
:1049A000E66E000EDA20E66E030EE66EEFEC13F014
:1049B000E552E552E552E552285001E0D5D0DF043A
:1049C0003FE1D950010FE96EDACFEAFFEE50ED106A
:1049D00017E10101010EF46F0101F56B000EE66EA7
:1049E000E66A000EE66EE66AB6CEE6FF000EE66EFA
:1049F000E66AABEC34F0456E070EE15E455016D02A
:104A0000D950010FE96EDACFEAFF010EEE1801E18D
:104A1000ED5006E10101F46B0101010EF56F06D0C6
:104A20000101010EF46F0101010EF56F000EE66E3B
:104A3000E66AE9C1E6FF05DBE552E552E55281D0C1
:104A4000020EDF5C15E1D950010FE96EDACFEAFF03
:104A5000EE50ED100AE10101010EE86F959E959A66
:104A6000949295989690959C02D00101E86B69D03C
:104A7000040EDF5C07E1010EDBCFB0FE020EDBCFE0
:104A8000B1FE5FD0050EDF5C07E1010EDBCFAEFEAD
:104A9000020EDBCFAFFE55D0080EDF5C16E1D95019
:104AA000010FE96EDACFEAFF180ED880EE54000E3F
:104AB000ED5407E2180EF36E010EF3CFDBFF020E8A
:104AC000DB6A010EDBCFAAFE3CD0090EDF5C16E1EB
:104AD000D950010FE96EDACFEAFF060ED880EE5406
:104AE000000EED5407E2060EF36E010EF3CFDBFF6E
:104AF000020EDB6A010EDBCFABFE23D00A0EDF5CB9
:104B00000DE1010EDBCFB2FE020EDBCFB3FE010ED4
:104B1000DBCFB4FE020EDBCFB5FE13D00B0EDF5C95
:104B200007E1010EDBCFB2FE020EDBCFB3FE09D0F0
:104B30000C0EDF5C06E1010EDBCFB4FE020EDBCF14
:104B4000B5FE0D0EDF5C0EE1D950010FE96EDACF34
:104B5000EAFFEE50ED1004E00101010EF06F02D00B
:104B60000101F06B36EC0BF0030EE15C02E2E16A4E
:104B7000E552E16EE552E7CFD9FF1200D9CFE6FF4B
:104B8000E1CFD9FF060EE126020EDB6A030EDB6AD7
:104B9000040EDB6A050EDB6AE66AD9CFE6FFDACFE0
:104BA000E6FF030EE66EEFEC13F0E552E552E55238
:104BB000E552E66AD950020FE66E000EDA20E66E84
:104BC000020EE66EEFEC13F0E552E552E552E552C7
:104BD000010EE66ED950040FE66E000EDA20E66E86
:104BE000020EE66EEFEC13F0E552E552E552E552A7
:104BF000285001E017D0040EDBCFE6FF050EDBCF17
:104C0000E6FF020EDBCFE6FF030EDBCFE6FFDECFD3
:104C1000E6FFDDCFE6FF10D8456E060EE15E45509B
:104C200036EC0BF0060EE15C02E2E16AE552E16E61
:104C3000E552E7CFD9FF1200D9CFE6FFE1CFD9FF88
:104C40001A5001E1FDD7D950FB0FE96EFF0EDA20B3
:104C5000EA6EEE50ED101CE1D950F90FE96EFF0E2F
:104C6000DA20EA6EEE50ED1013E10101020E996FA9
:104C7000190E396E3A6AFD0EDBCF3EF0FE0EDBCF29
:104C80003FF03CEC38F037C0A3F138C0A4F1F3D0CA
:104C9000010E0101A36FA46B0101A26B8D908B9299
:104CA000FB0EDBCF45F0FC0EDBCF46F00001800EA3
:104CB000461415E0020E0101A2110101A26F39682C
:104CC0003A68FB0EDBCF3EF0FC0EDBCF3FF00FEC83
:104CD00038F0FB0E37C0DBFFFC0E38C0DBFFF90EEF
:104CE000DBCF45F0FA0EDBCF46F00001800E461414
:104CF00015E0080E0101A2110101A26F39683A689E
:104D0000F90EDBCF3EF0FA0EDBCF3FF00FEC38F0C0
:104D1000F90E37C0DBFFFA0E38C0DBFFFD0EDBCF2C
:104D200049F0FE0EDBCF4AF04B6A4C6A190E3C6E1E
:104D30003D6A3E6A3F6A49C037F04AC038F04BC00E
:104D400039F04CC03AF0E4EC38F033C049F034C0EC
:104D50004AF035C04BF036C04CF0FB0EDBCF45F0CF
:104D6000FC0EDBCF46F0476A486A46AE02D0476881
:104D700048680F0ED8904536463647364836E8061E
:104D8000F9E145C037F046C038F047C039F048C0B7
:104D90003AF049C03CF04AC03DF04BC03EF04CC038
:104DA0003FF042EC39F037C09AF138C09BF1010E68
:104DB00001019A27000E01019B23FB0EDBCF9EF120
:104DC000FC0EDBCF9FF1FD0EDBCF49F0FE0EDBCFFB
:104DD0004AF04B6A4C6A190E3C6E3D6A3E6A3F6A65
:104DE00049C037F04AC038F04BC039F04CC03AF0F7
:104DF000E4EC38F033C049F034C04AF035C04BF031
:104E000036C04CF0F90EDBCF45F0FA0EDBCF46F0A2
:104E1000476A486A46AE02D0476848680F0ED89085
:104E20004536463647364836E806F9E145C037F09C
:104E300046C038F047C039F048C03AF049C03CF0AD
:104E40004AC03DF04BC03EF04CC03FF042EC39F060
:104E500037C09CF138C09DF1010E01019C27000E66
:104E600001019D23F90EDBCFA0F1FA0EDBCFA1F1FA
:104E70000101010E996F1A6AE552E7CFD9FF1200BE
:104E8000E9C145F0466A45BE466845C0E6FF46C0F2
:104E9000E6FFFE0E476E6A0E486E496A47C0E6FF9F
:104EA00048C0E6FF49C0E6FFC3EC37F04A6E050E86
:104EB000E15E4A5036EC0BF01200D9CFE6FFE1CFAD
:104EC000D9FF020EE126F40EDE6E010EDD6E010E3C
:104ED000E66ED9CFE6FFDACFE6FF030EE66EEFEC23
:104EE00013F0E552E552E552E552285001E019D0A1
:104EF0000101E9050AE1DECFE6FFDDCFE6FFE66A64
:104F0000A0D8E552E552E5520AD0DECFE6FFDDCF6C
:104F1000E6FF010EE66E95D8E552E552E55236EC15
:104F20000BF0020EE15C02E2E16AE552E16EE5524D
:104F3000E7CFD9FF1200D9CFE6FFE1CFD9FF050EA9
:104F4000E126DF6A010EDB6A020EDB6A010EF36EF8
:104F5000030EF3CFDBFFE66AD9CFE6FFDACFE6FF39
:104F6000010EE66EEFEC13F0E552E552E552E55224
:104F7000010EE66ED950010FE66E000EDA20E66EE5
:104F8000030EE66EEFEC13F0E552E552E552E55202
:104F9000010EE66ED950030FE66E000EDA20E66EC3
:104FA000010EE66EEFEC13F0E552E552E552E552E4
:104FB000E76E040EE7CFDBFF285001E038D0030E88
:104FC000DB50070805E2010EF36E030EF3CFDBFFA3
:104FD000DF50010802E2010EDF6E030EDB50030F0B
:104FE0000E01B65D16E0000EE66EE66A000EE66E95
:104FF000E66AB6CEE6FF000EE66EE66AABEC34F08B
:10500000456E070EE15E4550030EDB50030F0E01A7
:10501000B66F010EDBCFE6FF020EDBCFE6FFDFCF80
:10502000E6FF0FD8E552E552E55236EC0BF0050EDF
:10503000E15C02E2E16AE552E16EE552E7CFD9FFB9
:105040001200D9CFE6FFE1CFD9FF040EE126FE0E14
:10505000DB040BE1AECEDEFFAFCEDDFF020EB2CE43
:10506000DBFF030EB3CEDBFF0AD0B0CEDEFFB1CE46
:10507000DDFF020EB4CEDBFF030EB5CEDBFFFC0E70
:10508000DBCFE6FFFD0EDBCFE6FF020EDBCFE6FF58
:10509000030EDBCFE6FFB6CEE6FFDECFE6FFDDCFC9
:1050A000E6FFABEC34F0456E070EE15E4550040EB2
:1050B000E15C02E2E16AE552E16EE552E7CFD9FF39
:1050C0001200D9CFE6FFE1CFD9FF050EE126E66A4F
:1050D000D9CFE6FFDACFE6FF010EE66EEFEC13F074
:1050E000E552E552E552E552E76E040EE7CFDBFFED
:1050F000040EDB5030E1285001E05BD00101E851A3
:1051000024E0DF5000081FE28D90DF0403E18D846E
:105110008D82898C020EDF5C03E18D848D82899CF7
:10512000030EDF5C03E18D948D82899C040EDF5CAD
:1051300003E18D848D92899C050EDF5C03E18D94E3
:105140008D92899C01D08D8006D0DF50000802E24C
:105150008D9001D08D80010EE66ED950010FE66E64
:10516000000EDA20E66E010EE66EEFEC13F0E5526B
:10517000E552E552E552E76E040EE7CFDBFF040E81
:10518000DB5015E1285001E014D00101E85108E09E
:10519000010EDB50000802E28B9201D08B8207D017
:1051A000010EDB50000802E28C9C01D08C8C36ECA6
:1051B0000BF0050EE15C02E2E16AE552E16EE552B8
:1051C000E7CFD9FF1200FE0E0101EA5DFF0EEB5999
:1051D000FF0EEC59FF0EED5906E20101EA2B000E1D
:1051E000EB23EC23ED2336EC0BF012000101EA5126
:1051F000EB11EC11ED1106E00101EA07000EEB5B8B
:10520000EC5BED5B36EC0BF01200D9CFE6FFE1CFA3
:10521000D9FF050EE126E66AD9CFE6FFDACFE6FF31
:10522000070EE66EEFEC13F0E552E552E552E5525B
:10523000E76E040EE7CFDBFF040EDB500BE1DFCFA0
:10524000EAF1010EDBCFEBF1020EDBCFECF1030E46
:10525000DBCFEDF136EC0BF0050EE15C02E2E16A2A
:10526000E552E16EE552E7CFD9FF1200EAC1E6FF51
:10527000EBC1E6FFECC1E6FFEDC1E6FFF50E456EC2
:105280006A0E466E476A45C0E6FF46C0E6FF47C065
:10529000E6FFC3EC37F0486E070EE15E485036EC8F
:1052A0000BF01200E66AEE0EE66E010EE66E010EDF
:1052B000E66EEFEC13F0E552E552E552E552285068
:1052C00001E002D036EC0BF01200EEC145F0466A68
:1052D00045BE466845C0E6FF46C0E6FFEE0E476E97
:1052E0006A0E486E496A47C0E6FF48C0E6FF49C0FB
:1052F000E6FFC3EC37F04A6E050EE15E4A5036EC2D
:105300000BF01200EFC145F0466A45BE466845C045
:10531000E6FF46C0E6FFE80E476E6A0E486E496A31
:1053200047C0E6FF48C0E6FF49C0E6FFC3EC37F0E0
:105330004A6E050EE15E4A500101EF6B36EC0BF050
:105340001200D9CFE6FFE1CFD9FF040EE126DE6AD5
:10535000DD6A020EDB6A030EDB6AC26AA40EC16E4E
:105360009E9C9F9CC28001010A0EF16F0101F151C8
:1053700001E0FCD7C282C2B2FED7C450476E47C01C
:1053800048F0476AC35000014724456E000E48208C
:10539000466E45C0DEFF46C0DDFF2D0EC26E010128
:1053A0000A0EF16F0101F15101E0FCD7C282C2B2D5
:1053B000FED7C450476E47C048F0476AC35000014B
:1053C0004724456E000E4820466E020E45C0DBFFA6
:1053D000030E46C0DBFF020EDBCFE6FF030EDBCF82
:1053E000E6FFDECFE6FFDDCFE6FFDC0E456E6A0EA0
:1053F000466E476A45C0E6FF46C0E6FF47C0E6FF87
:10540000C3EC37F0486E070EE15E485036EC0BF007
:10541000040EE15C02E2E16AE552E16EE552E7CF9B
:10542000D9FF1200D9CFE6FFE1CFD9FF030EE12665
:10543000DF6A010EDB6A040EF36E020EF3CFDBFFB0
:10544000E66AD9CFE6FFDACFE6FF010EE66EEFECB3
:1054500013F0E552E552E552E552010EE66ED950E1
:10546000010FE66E000EDA20E66E030EE66EEFEC3C
:1054700013F0E552E552E552E552285001E057D0CD
:10548000D950010FE96EDACFEAFFFF0ED880EE5453
:10549000030EED5420E3010EDBCFF2F1020EDBCF61
:1054A000F3F1CB680101F26B020EF36FFC0ECA142C
:1054B0000009CA6E9D920F0152810F015293F00EA6
:1054C000BA140C09BA6E3F0EBA140009BA6E0E0176
:1054D0000E0ECC6FCA84DF5024E0F2C145F0F3C158
:1054E00046F0D89046324532D89046324532455043
:1054F000BB6EF2C147F0F3C148F0040ED8904736B6
:105500004836E804FBE1300E4716000E4816CF0E71
:10551000BA1400014710456E48C046F04550BA6EB7
:1055200004D0BB6ACF0EBA14BA6E36EC0BF0030E81
:10553000E15C02E2E16AE552E16EE552E7CFD9FFB4
:1055400012001200000EE66EE66A000EE66EE66AD3
:105550001A50456E466A45BE466845C0E6FF46C0DD
:10556000E6FFCE0E476E6A0E486E496A47C0E6FFF8
:1055700048C0E6FF49C0E6FFC3EC37F04A6E090EAB
:06558000E15E4A5012003A
:0A558600FFEC2FF0FB0EDBCFF3FF6C
:10559000DB06F35000090AE04DEC30F0FA0EB8ECEF
:1055A00030F0F3E1461CF1E1010E01D0000E2EEFC8
:1055B00030F0FFEC2FF03B0EE12402E3E168E6520D
:1055C000E16E010EDB6A020EDB6AF90EDBCFF6FF3D
:1055D000FA0EDBCFF7FFFB0EDBCFF8FF0800F5502C
:1055E000DF6EDF5002E152EF2FF0250EDF5C02E0AC
:1055F00045EF2FF0030EDB6A040EDB6A050EDB6A53
:10560000060EDB6A070EDB6A67EC2FF02D0EDF5CFF
:105610000CE02B0EDF5C09E0200EDF5C06E0230EC1
:10562000DF5C03E0300EDF5C1AE1DF50300A14E08B
:10563000130A0FE0030A0AE00B0A05E0060AE4E198
:10564000030EDB80E1D7030EDB82DED7030EDB84A3
:10565000DBD7030EDB86D8D7030EDB88D5D72A0E1F
:10566000DF5C1BE163EC2FF0B1EC2FF010E0030ED8
:10567000DB8039683A68130EDBCF3EF0140EDBCFC7
:105680003FF00FEC38F0040E37C0DBFF03D0130EF1
:105690009AEC2FF067EC2FF00BD0090EDB6A08ECC8
:1056A00030F003E07CEC30F0FAD7090E9AEC2FF0E2
:1056B000030EDBB0DB982E0EDF5C1BE167EC2FF0F6
:1056C0002A0EDF5C0BE163EC2FF0B1EC2FF003E16D
:1056D000130EECEC2FF067EC2FF00BD0090EDB6A09
:1056E00008EC30F003E07CEC30F0FAD7090EECEC7B
:1056F0002FF0680EDF5C07E167EC2FF0680EDF5CCF
:105700001DE1030E18D0740EDF5C17E07A0EDF5C2B
:1057100014E0480EDF5C06E0540EDF5C03E05A0E36
:10572000DF5C02E1020E07D06C0EDF5C03E06A0E64
:10573000DF5C04E1010E3FEC30F0C9DBDF506E0AA4
:1057400001E17FD31E0A01E192D1200A01E18FD14C
:105750003F0A01E149D11A0A01E146D10D0A01E1EE
:1057600043D1200A01E140D13A0A01E13DD1200AAA
:1057700001E13AD1260A01E135D10D0A01E132D128
:105780001A0A01E1D9D0200A4AE0300A1FE0460A8D
:105790000EE0250A01E083D3D950F90FE96EFF0E20
:1057A000DA20EA6E010EEE5E000EEE5AEE5A4DEC75
:1057B00030F0250EE66E95DB03E1461C01E169D36E
:1057C00049EC30F001E26BD3DB2A69D3080EDB6AC7
:1057D000040EDB50010806E2040EDB0411EC30F08D
:1057E000DB508BDB080EDB5009E0030EDB50010BB6
:1057F00005E172DB01E04DD3080EDB6A64DBEFCF1D
:10580000DFFFC1EC30F003E1461C01E142D349EC7B
:1058100030F001E3DB2A60DB01E141D33AD3070E2C
:10582000DB5002080FE18DEC30F0030E54EC30F049
:105830000E0EEECFDBFF0F0EEECFDBFF100EEECF26
:10584000DBFF20D0F70EDBCF48F0F80EDBCF49F0BE
:10585000020E485E000E495AF70E48C0DBFFF80EF4
:1058600049C0DBFF48C0E9FF49C0EAFF44EC30F023
:10587000476A0E0E45C0DBFF0F0E46C0DBFF100E61
:1058800047C0DBFF0E0EDBCFE6FF0F0EDBCFE6FFE0
:10589000100EDBCFE6FF9EEC37F0E552E552E55205
:1058A000130E38C0DBFF140E39C0DBFF060EDB50D1
:1058B00005E0130E88EC30F001E26ADBACEC30F06E
:1058C00002E2130E37DB6FEC30F006E0040E88ECDA
:1058D00030F002E2050E2EDB030EDBB005D0FCDA61
:1058E00001E0D7D2080EDB6A090EDB6A0E0EDBCFB1
:1058F000F6FF0F0EDBCFF7FF100EDBCFF8FF08002F
:10590000F550DF6EDF5014E0B2EC30F011E2C1EC84
:1059100030F003E1461C01E1BCD2BBDB01E3DB2A32
:10592000090EDB2AD9500E0FE96E000ECBDBE7D74C
:10593000D3DA01E1B4D2ADD2C6DA110EEECFDBFF7D
:10594000120EEDCFDBFF110EDBCFE6FF120EDBCF29
:10595000E6FF90EC37F0E552E552130EF3CFDBFF94
:10596000140EF4CFDBFF060EDB5004E0130ED0DB89
:1059700001E20EDBACEC30F002E2130EDBDAAFDB5F
:1059800005E0040EC5DB02E2050ED4DA030EDBB03F
:1059900005D0A2DA01E07DD2080EDB6A090EDB6ACF
:1059A000110EDBCFE9FF120EDBCFEAFFEFCFDFFFF7
:1059B000DF5014E0D7DB12E2E4DB03E1461C01E137
:1059C00068D267DB01E3DB2A090EDB2A110EDB2A32
:1059D000DBCFE9FF120EE8E3DB2AE6D77DDA01E14F
:1059E0005ED257D2030EDB8E070EDB0410E195DB8F
:1059F000040E5ADB0A0EEECFDBFF0B0EEECFDBFF01
:105A00000C0EEECFDBFF0D0EEECFDBFF6CD0070EE2
:105A1000DB5003082CE1030EDBAE0DD0B2DA020E30
:105A200076DAEFCF45F0466A476A486A45AE39D024
:105A30004668476835D0F70EDBCF46F0F80EDBCF6F
:105A400047F0020E465E000E475AF70E46C0DBFFD7
:105A5000F80E47C0DBFF46C0E9FF47C0EAFFEFCFC3
:105A600045F00A0E45C0DBFF0B0EDB6A38D0070E8F
:105A7000DB50020809E1030EDBAE04D059DB47AE70
:105A800010D00ED055DB0DD0030EDBAE12D079DA7C
:105A9000020E3DDAF9DA476A486A46AE02D0476834
:105AA0004868E2DA0C0E47C0DBFF0D0E48C0DBFF92
:105AB0001AD0F70EDBCF47F0F80EDBCF48F0020E1E
:105AC000475E000E485AF70E47C0DBFFF80E48C08D
:105AD000DBFF47C0E9FF48C0EAFFD6DAC5DA0C0EA3
:105AE000DB6A0D0EDB6A060EDB5005E1010EF36E7C
:105AF000050EF3CFDBFF150EDB6A160EDB6AD950FD
:105B0000370F456E000EDA20466E390E45C0DBFFBA
:105B10003A0E46C0DBFF380EDB6A080EDB6A0A0E5F
:105B2000AEDADF50780A12E0200A10E0280A0CE012
:105B3000200A0AE03F0A06E00D0A02E0200A08E116
:105B4000020E05D0080E03D0080EDF26100E97DADD
:105B5000030EDBBE02D0DB92DB94DB50800B24E033
:105B60008ADAD890030EEB50000A08E6000EEE5CCD
:105B7000000EEE58000EEE58000EEE5815E213DA45
:105B80003C683D683E683F68E4EC38F00A0E33C07C
:105B9000DBFF0B0E34C0DBFF0C0E35C0DBFF0D0E40
:105BA00036C0DBFF2D0E08D0030EDBA202D02B0E79
:105BB00003D0DBA408D0200EF36E170EF3CFDBFF6B
:105BC000150EDB2A02D0170EDB6A050EDB5003E14F
:105BD000B7D901E189D05A0E456E730E466E000E9C
:105BE000476E070EDBCF48F0496A4A6A4B6A48C0E5
:105BF0003CF049C03DF04AC03EF04BC03FF0D3D925
:105C000042EC39F045503324F36E46503420F46EA4
:105C100047503520F86EF4CFF7FFF3CFF6FF0800BA
:105C2000090EF5CFDBFF580EDF5C0FE1610EF36E5E
:105C3000090E7BD90AE3200E456E090EDBCFE7FF84
:105C40004550E75E090EE7CFDBFF070EDBCF45F0DF
:105C5000466A476A486A0FDA45C03CF046C03DF0E4
:105C600047C03EF048C03FF0EECF37F0EECF38F0FF
:105C7000EECF39F0EFCF3AF042EC39F03AC0EDFF19
:105C800039C0EDFF38C0EDFF37C0EFFF390EDBCF75
:105C9000E9FFDB063A0EDBCFEAFF01E2DB06090E85
:105CA000DBCFEFFF150EDB2A4BD995E1030EDBA608
:105CB0001DD06F0EDF5C06E1C1D918E3150EDB289D
:105CC0005BDA14D0780EDF5C09E0580EDF5C06E08A
:105CD000620EDF5C03E0420EDF5C08E1020EF36E51
:105CE000160EF3CFDBFF02D0150EDB6A030EDB507E
:105CF000100B0EE0040EDBCF45F0050EDB50D88014
:105D0000455406E2060EDB5003E1040EDB5034DAA4
:105D100095D90AE2050EDBCFE7FF150EDB50E75EF3
:105D2000050EE7CFDBFF02D0050EDB6A040EDBCFEA
:105D300045F0160E45D9D880455414E2160EDBCF37
:105D4000E6FF150EDBCFE6FF040EDBCFE6FF050E08
:105D5000DB50E552E75CE552D880E754E552D88045
:105D6000E7545FD9030EDB50010B0BE1080EDB504B
:105D700008E0B2D801E08DD0080EDB50BED8080E86
:105D8000DB6A170EDB5007E088D9170EF1D903E163
:105D9000461C01E17ED0160EDB5016E07ED9300E97
:105DA000E66E9FD802E1461C74E077D9DFCFE6FFAC
:105DB000A2EC38F0E552E552E552F4CF46F000018E
:105DC000F31C02E1461C65E0050EDBCF45F0160E24
:105DD000DB50D880455409E2050EDBCFE7FF160EF5
:105DE000DB50E75E050EE7CFDBFF300EE66E050EFB
:105DF000CBD94FE1390EDB2ADBCFE9FF3A0E01E3C5
:105E0000DB2ADBCFEAFF090EEFCFDBFFDB500EE032
:105E100044D9090EADD902E1461C3BE0390EDB2A1C
:105E2000DBCFE9FF3A0EEDE3DB2AEBD755D831E1C2
:105E3000160EDBCFE6FF080EC3D8E552E7245DD887
:105E40002ED0070EDB50030A1CE0010A14E0030AFF
:105E500007E07BD9DBCFEEFF020EDBCFEDFF1FD0DB
:105E6000F5D84A6A48AE02D049684A682CD8BCD8EE
:105E70004AC0EEFF14D0EAD848BE496824D8B4D846
:105E80000ED063D9DBCFEFFF0AD07BD905E1461CEA
:105E900003E1F368F46810D0FCD801E3DB2A79D978
:105EA000EEEF2AF0010EDBCF45F0020EDBCF46F01D
:105EB00045C0F3FF46C0F4FF3B0EE15C02E2E16A3D
:105EC000E552E16ECBD029D9020E54EF30F061D902
:105ED0000800F550DF6E1200200EE66E080EC4EFCB
:105EE00030F0A2EC38F0E552E552E552F3CF45F040
:105EF000F4CF46F00001F31C1200456E466AD950FB
:105F0000010F4DD94550EE264650ED221200495E54
:105F1000000E4A5AF70E49C0DBFFF80E4AC0DBFFFD
:105F200049C0E9FF4AC0EAFF1200DBCFF4FFF3509B
:105F3000F45C1200DB50E76E040EE7CFDBFF1200CB
:105F40000A0EDBCF45F00B0EDBCF46F00C0EDBCF9D
:105F500047F00D0EDBCF48F0455046104710481073
:105F60001200130EEECFDBFF140EEDCFDBFF130E8E
:105F7000DBCF45F0140EDBCF46F00001800E461457
:105F80001200F70EDBCF49F0F80EDBCF4AF012001B
:105F9000050EDB50E66ED950130F01D9E552E750DC
:105FA000EE6EED6A12000A0EDBCF37F00B0EDBCF80
:105FB00038F00C0EDBCF39F00D0EDBCF3AF01200CB
:105FC000DBCFE6FF150EDBCFE6FF050EDB50E5521B
:105FD000E724E552E7241200DB50CED8010EF36E21
:105FE000060EF3CFDBFF1200EE50EFCFEAFFE96EB3
:105FF00047C0EEFF48C0EEFF49C0EEFF1200D9CF08
:10600000E6FFDACFE6FFE1CFD9FFE2CFDAFF1200F9
:10601000DFCFE6FFE66A30EC39F0E552E552F350A7
:106020001200E76E080EE7CFDBFF1200EECF45F05F
:10603000EECF46F0EFCF47F0486A1200050EDBCFF7
:1060400045F0150EDB50D88045541200010EDBCF11
:1060500047F0020EDBCF48F0496A1200E552E5CF67
:10606000DAFFE7CFD9FF12000A0E45C0DBFF0B0EA7
:1060700046C0DBFF1200D9500A0FCFEF30F0F36EAD
:10608000070EF3CFDBFF1200EECF45F0EFCF46F067
:106090001200010EDB2A020E1200FC0EDBCFE6FF1F
:1060A000FD0EDBCFE6FF1200455E000E465AF70EEE
:1060B00045C0DBFFF80E46C0DBFF45C0E9FF46C028
:1060C000EAFF1200DA20EA6EEF2AEECFF6FF000EAA
:1060D000EF22EECFF7FFEF22EECFF8FF1200040E13
:1060E000DBCFE6FF130EDB50E552E75C9ADFDB50B7
:1060F00004DF060EDB501200090EDB500A0DF350D0
:10610000DF24D00FE76E090EE7CFDBFF67EF2FF03C
:10611000DB50F36E050E95EF2FF0F70EDBCF45F059
:10612000F80EDBCF46F01200DFCFE6FF71EF2FF065
:1061300028DF030EECDE16EF30F0C3EC2AF0E55258
:10614000E552E552E55200091200BDDEEE50EFCFF8
:10615000EAFFE96E010E1200130EDB50F36E040E1F
:1061600095EF2FF0040EDB50F36E090E95EF2FF034
:10617000DBCFE6FF71EF2FF0E76E050EE7CFDBFF19
:1061800012008BDF94EF30F0DBCFE6FF86DF9DEF70
:1061900030F0D950F90FE96EFF0E62EF30F0E96E82
:0861A000000EDA20EA6E120085
:0861A800040130511F0B010836
:1061B00001E057D004013051600BE842E842E84268
:1061C000E842E842010801E04CD00401345104E007
:1061D0000401340501E045D004013151220A3BE0BD
:1061E000030A2CE0010A1BE0210A11E0010A01E088
:1061F00037D00601A00EBD6F060EBE6F080E060159
:10620000C06FC16B0601BF810601BF8F2AD0060196
:10621000A00EBD6F060EBE6F0601BF8F22D036C422
:10622000C5F637C4C6F60601800EC26F060EC36FF0
:106230000601C76BC86B0601C48F13D00601800E20
:10624000BD6F060EBE6F070E0601C06FC16B060163
:10625000C10EBF6F06D032C49BF60601BF8F01D0BE
:1062600000D012000601806B4B0E816F826B836B36
:106270000601846B0601856B0601080E866F060118
:106280008F6B1A0EE66E010EE66EF4EC19F0E55215
:10629000E5521E0EE66E020EE66EF4EC19F0E552C3
:1062A000E552400EE66E400EE66E060EE66EE66ABB
:1062B000020EE66E2BEC1AF0456E050EE15E4550BF
:1062C000F3CF97F6F4CF98F60601996B9A6B060117
:1062D000906B1200D9CFE6FFE1CFD9FFFD0EDBCFE7
:1062E00039F0FE0EDBCF3AF0050E391801E13A50D5
:1062F00001E032D0FB0EDBCF45F0FC0EDBCF46F0E9
:1063000006019751451802E19851461813E1400ED5
:10631000E66E400EE66E060EE66EE66A020EE66E6B
:106320002BEC1AF0456E050EE15E4550F3CF97F663
:10633000F4CF98F6FB0EDBCF45F0FC0EDBCF46F03A
:1063400006019951451802E19A51461804E10601E7
:10635000906B0601956B02D0000E02D0010E00D0AA
:10636000E552E7CFD9FF1200D9CFE6FFE1CFD9FF41
:1063700006018F6B06019751981102E1000E08D0BB
:1063800097C6E9FF98C6EAFFEF50800B01E0010EC7
:1063900000094AE1FC0EDBCF45F097C6E9FF98C63D
:1063A000EAFFEE52EF50D880455408E297C6E9FF65
:1063B00098C6EAFFEE52FC0EEFCFDBFF06018F6BB3
:1063C000FC0EDB5006018F5D1CE206018F51EA6A6C
:1063D000400FE96E060EEA22EF50E66E06018F517D
:1063E000E76EFD0EDBCFE9FFFE0EDBCFEAFFE750E5
:1063F000E926000EEA22E552E750EF6E06018F2BE8
:10640000DFD7400EE66E400EE66E060EE66EE66ADA
:10641000020EE66E2BEC1AF0456E050EE15E45505D
:10642000F3CF97F6F4CF98F606018F5100D0E552DE
:10643000E7CFD9FF1200D9CFE6FFE1CFD9FF0601A0
:1064400090510FE1FD0EDBCF91F6FE0EDBCF92F601
:10645000FC0EDBCF95F60601010E966F0601010ECC
:10646000906FE552E7CFD9FF1200D9CFE6FFE1CF19
:10647000D9FF030EE1260601905101E030D0DF6A1A
:10648000FD0EDBCF39F0FE0EDBCF3AF0DE5239C025
:10649000DEFF3AC0DDFFDD52DF2ADF50456E466A7F
:1064A000FF0E451801E1465001E10BD0010EDBCF94
:1064B000E9FFDB2A020EDBCFEAFF01E3DB2AEF5024
:1064C000EBE1FD0EDBCF91F6FE0EDBCF92F6DFCFD8
:1064D00095F60601010E966F0601010E906F030EF0
:1064E000E15C02E2E16AE552E16EE552E7CFD9FFF5
:1064F0001200D9CFE6FFE1CFD9FF030EE126060156
:10650000905101E030D0DF6AFD0EDBCF39F0FE0E96
:10651000DBCF3AF0DE5239C0DEFF3AC0DDFFDD529C
:10652000DF2ADF50456E466AFF0E451801E14650EE
:1065300001E10CD0010EDBCFF6FFDB2A020EDBCF30
:10654000F7FF01E3DB2A0800F550EAE1FD0EDBCF9F
:1065500091F6FE0EDBCF92F6DFCF95F60601966B35
:106560000601010E906F030EE15C02E2E16AE55262
:10657000E16EE552E7CFD9FF1200D9CFE6FFE1CFB8
:10658000D9FF020EE126060199519A1102E1000E8F
:1065900008D099C6E9FF9AC6EAFFEF50800B01E0E8
:1065A000010E000901E098D0030E0601905D02E1A2
:1065B0000601906B0601905101E18ED0020E06019A
:1065C000905D16E1E66A000EE66EE66A010EE66E82
:1065D000020EE66E2BEC1AF0456E050EE15E45509C
:1065E000F3CF99F6F4CF9AF60601030E906F74D0AC
:1065F0000601900571E1400E456E466A060195510F
:10660000455C000E465803E2400EDF6E02D095C690
:10661000DFFFDF500601955D0601956F0601000E54
:10662000936F060E946F010EDFCFDBFF06019651CC
:106630001AE1010EDB5016E091C6F6FF92C6F7FF95
:106640000800F55093C6E9FF94C6EAFFEF6E060115
:10665000932B000E94230601912B000E9223010E22
:10666000DB06E7D718D0010EDB5015E091C6E9FF35
:1066700092C6EAFFEF5093C6E9FF94C6EAFFEF6EB9
:106680000601932B000E94230601912B000E9223FA
:10669000010EDB06E8D7060195510AE1400EDF5CEA
:1066A00004E10601020E906F03D00601030E906F05
:1066B000DFCFE6FF000EE66E060EE66E010EE66E1A
:1066C000020EE66E2BEC1AF0456E050EE15E4550AB
:1066D000F3CF99F6F4CF9AF6020EE15C02E2E16A9A
:0C66E000E552E16EE552E7CFD9FF120051
:0466EC00D9CFE6FF1D
:1066F000E1CFD9FFE6520E01006B0E01A96BDF6AF4
:10670000180EDF5C2AE2EA6ADF34FE0BEA36E96E35
:10671000010EE9260E0EEA22EE6AED6ADF50EA6A01
:10672000310FE96E0E0EEA22EF6AEA6ADF34FE0BE1
:10673000EA36E96E490EE9260E0EEA22EE6AED6AA5
:10674000EA6ADF34FE0BEA36E96E790EE9260E0EB0
:10675000EA22EE6AED6ADF2AD3D70E01C60EAC6FCD
:106760000E0EAD6F3F0E79140009796ECF0E7914BD
:106770000009796E79827B6A7A6A79900F01528179
:106780000F015293F00EB4140909B46E0E01080EF5
:10679000AA6F0E01030EAB6F0E01200EB06F4E0EEE
:1067A000B16F0E01800EAE6F3E0EAF6F0E01040E84
:1067B000B66F0E01900EB26F010EB36F0E01900E08
:1067C000B46F010EB56F000EE66EE66A010EE66E5E
:1067D00021EC28F0E552E552E552E552E552E7CFCB
:1067E000D9FF1200D9CFE6FFE1CFD9FFE652DF6A29
:1067F000180EDF5C10E2DF50EA6A310FE96E0E0E10
:10680000EA22EFCF45F0FE0EDB50455C02E1DF28C7
:1068100014D0DF2AEDD7DF6A180EDF5C0CE2DF5000
:10682000EA6A310FE96E0E0EEA22EF5002E1DF282C
:1068300004D0DF2AF1D7000E00D0E552E552E7CFB1
:10684000D9FF1200D9CFE6FFE1CFD9FF080EE1262C
:10685000DF6A010EDB6A020EDB6A030EDB6A040EDE
:10686000DB6A050EDB6A060EDB6A070EDB6A010EC9
:10687000E66ED950010FE66E000EDA20E66E030ECA
:10688000E66EEFEC13F0E552E552E552E552010EEB
:10689000E66ED950030FE66E000EDA20E66E010EAA
:1068A000E66EEFEC13F0E552E552E552E552010ECB
:1068B000E66ED950040FE66E000EDA20E66E030E87
:1068C000E66EEFEC13F0E552E552E552E552010EAB
:1068D000E66ED950060FE66E000EDA20E66E030E65
:1068E000E66EEFEC13F0E552E552E552E552285022
:1068F00001E027D0DF50180802E2288C22D0030ED6
:10690000DB50180802E2288C1CD0060EDBCFE6FF15
:10691000070EDBCFE6FF040EDBCFE6FF050EDBCF75
:10692000E6FF030EDBCFE6FF010EDBCFE6FF020E34
:10693000DBCFE6FF10D8456E070EE15E455036EC22
:106940000BF0080EE15C02E2E16AE552E16EE5520D
:10695000E7CFD9FF1200D9CFE6FFE1CFD9FF020E72
:10696000E126F29CFC0EDBCFE6FF3CDFE552E76E52
:10697000010EE7CFDBFF010EDB5003E1F28C000ECE
:106980009AD0D950FD0FE96EFF0EDA20EA6EEE5074
:10699000ED103FE1010EDB04EA6A310FE96E0E0EE5
:1069A000EA22EF500E01EA6AAC25E96EAD51EA2207
:1069B000EF6A010EDB04E96EEA6AD890E936EA363E
:1069C000790EE9260E0EEA22EE6AED6A010EDB046C
:1069D000E96EEA6AD890E936EA36490EE9260E0EE3
:1069E000EA22EE6AED6A010EDB04EA6A310FE96E13
:1069F0000E0EEA22EF6A010EDB04E96EEA6AD89015
:106A0000E936EA36010EE9260E0EEA22EE6AED6A52
:106A10004ED0010EDB04456E0E01AA51455C47E2E3
:106A2000FC0EDB50180843E3FC0EDB50070802E1C4
:106A30000101F46B010EDB04E96EEA6AD890E936D5
:106A4000EA36010EE9260E0EEA22EE50ED1010E1B4
:106A5000E66AFC0EDBCFE6FFFFEC17F0E552E552ED
:106A6000E66AFC0EDBCFE6FF95EC17F0E552E55247
:106A70001A5001E1FDD70101030E996FF80EDBCF2B
:106A8000A3F1F90EDBCFA4F1010EDBCFA8F1FC0ED0
:106A9000DBCFA7F1FD0EDBCFA5F1FE0EDBCFA6F11C
:106AA000FA0EDBCFA9F1FB0EDBCFAAF11A6AF28C4A
:106AB000010EDB5000D0456E020EE15C02E2E16A9D
:0E6AC000E552E16E4550E552E7CFD9FF1200D6
:026ACE00514D28
:106AD0002C25692C25692C25690A0D00253034697F
:106AE0002C253034690D0A002531690D0A00253046
:106AF00033690D0A00253031306C750D0A002564AC
:106B00000A0D005374617475733D25690D0A0021E7
:106B100035204572723A204E65656420636F6D6D55
:106B200061206E6578742C20666F756E643A20273C
:106B30002563270D0A00506172616D383D25630D94
:106B40000A00506172616D373D25630D0A00506186
:106B500072616D363D256C750D0A00506172616D74
:106B6000353D256C640D0A00506172616D343D2520
:106B7000750D0A00506172616D333D25640D0A0088
:106B8000506172616D323D25640D0A005061726181
:106B90006D313D25640D0A0050492C2531750D0AD3
:106BA000004D522C253033750D0A002C25303475DC
:106BB000004100492C253033692C253033692C25C0
:106BC0003033692C253033692C253033690D0A00A8
:106BD0002138204572723A20556E6B6E6F776E20A9
:106BE000636F6D6D616E642027256325633A2532DE
:106BF00058253258270D0A002138204572723A2054
:106C0000556E6B6E6F776E20636F6D6D616E642075
:106C10002725633A253258270D0A0021372045726F
:106C2000723A204578747261207061726D6174658A
:106C3000720D0A002136204572723A20496E766143
:106C40006C696420706172616D7465722076616C2C
:106C500075650D0A002134204572723A204D697322
:106C600073696E6720706172616D657465722873F7
:106C7000290D0A002133204572723A2052582042D1
:106C80007566666572206F76657272756E0D0A00A4
:106C90002132204572723A2054582042756666654A
:106CA00072206F76657272756E0D0A002131204573
:106CB00072723A2043616E27742073746570207479
:106CC00068617420666173740D0A002130200D0A1A
:106CD000002008002573001B5B421B5B314B1B5BD4
:036CE0003047003A
:0C6CE40006D805EC19F033EC05F0FBD7E6
:106CF0001200D9CFE6FFE1CFD9FF020EE1260F0146
:106D000048690F014969600ED36E9B8C580EDE6E88
:106D1000020EDD6EDFCF45F0DF06010EDBCF46F061
:106D200001E2DB064550461001E0F4D7948E4DECAD
:106D300004F069EC18F0020EE15C02E2E16AE5524F
:106D4000E16EE552E7CFD9FF1200120012001200E7
:106D50001200D4EC30F01200120032EC31F01200CC
:106D60000601CB0523E10601CC0520E1EFDF6592AA
:106D70000601CC6B0E01100EB76F0E0EB86F0E0130
:106D8000B707000EB85B0E01B751B811F8E1658482
:106D90000E01080EB76F070EB86F0E01B707000E91
:106DA000B85B0E01B751B811F8E165941200D9CF64
:106DB000E6FFE1CFD9FFFD0EDBCF39F0FE0EDBCFD2
:106DC0003AF0050E391801E13A5039E0E86839180F
:106DD00002E17F0E3A1831E0030E391801E13A5012
:106DE0002AE0020E391801E13A5023E0010E391869
:106DF00001E13A501CE0740E391801E13A5015E0F7
:106E0000750E391801E13A500EE0730E391801E1A0
:106E10003A5007E0720E391801E13A5001E010D003
:106E200010D095DF0ED091DF0CD090DF0AD095DF27
:106E300008D092DF06D08DDF04D08ADF02D001D0E7
:0E6E400000D0010E00D0E552E7CFD9FF1200BE
:026E4E002A0E0A
:106E5000F66E000EF76E000EF86E01010900F55097
:106E6000FB6F0900F550FC6F03E1FB6701D03DD0DB
:106E70000900F550F66F0900F550F76F0900F5505D
:106E8000F86F09000900F550E96E0900F550EA6E47
:106E9000090009000900F550F96F0900F550FA6F73
:106EA00009000900F6CFFDF1F7CFFEF1F8CFFFF1B1
:106EB000F6C1F6FFF7C1F7FFF8C1F8FF0101F9537A
:106EC00002E1FA5307E00900F550EE6EF907F8E227
:106ED000FA07F9D7FDC1F6FFFEC1F7FFFFC1F8FFC2
:0C6EE0000101FB07000EFC5BBFD7120095
:046EEC00FE0EE3CFE4
:106EF000E9FFFF0EE3CFEAFFE9CFF3FFEACFF4FFAC
:106F0000FB0EE35003E1FC0EE35009E0FB0EE30649
:106F100002E2FC0EE306FD0EE350EE6EF1D7120026
:106F2000FE0EE3CFE9FFFF0EE3CFEAFFF36AF46A58
:106F3000EE5203E0F34AF42AFBD71200FF0EE3CF30
:106F4000F8FFE552FF0EE3CFF7FFE552FF0EE3CF68
:106F5000F6FFE552E66AE66AE66A0900F55209E0DC
:106F6000FD0EE32A05E1FE0EE32A02E1FF0EE32A0D
:106F7000F4D7FD0EE3CF38F0FE0EE3CF39F0FF0E6D
:066F8000E3CF3AF012001D
:0A6F8600D9CFE6FFDACFE6FFE1CF36
:106F9000D9FFE2CFDAFFE652E652E652E652D95086
:106FA000FB0F456EFF0EDA20466E45C0DEFFDD6E3C
:106FB000DECFE6FFDDCFE6FFFB0EDBCFE6FFFC0E0C
:106FC000DBCFE6FFFD0EDBCFE6FFB9CEE6FFBACEA4
:106FD000E6FFD9EC2AF0456E070EE15C02E2E16AB9
:106FE000E552E16E4550020EF3CFDBFF030EF4CF06
:106FF000DBFF020EDBCF45F0030EDBCF46F045C0D2
:10700000F3FF46C0F4FF040EE15C02E2E16AE552E0
:0E701000E16EE552E5CFDAFFE7CFD9FF1200BF
:02701E003AC076
:1070200044F039C043F039503E02F4CF38F0F3CF8A
:1070300037F03A503F02F4CF3AF0F3CF39F03E0246
:10704000F3503826F4503922E86A3A2243503F027E
:10705000F3503826F4503922E86A3A223FAE35EF31
:1070600038F04350395E44503A5A44AE000C3E501A
:10707000395E3F503A5A000C39C043F039503E0255
:10708000F4CF38F0F3CF37F03A503F02F4CF3AF074
:10709000F3CF39F03E02F3503826F4503922E86A33
:1070A0003A2243503F02F3503826F4503922E86A1E
:0470B0003A22000C74
:0C70B4001201000202000040D80492FD0E
:1070C00082010102000109024300020100C03209ED
:1070D0000400000102020100052400100104240242
:1070E00002052406000105240100010705810308AB
:1070F000000209040100020A000000070502024024
:10710000000007058202400000040309041803532D
:1071100000630068006D0061006C007A0048006147
:10712000007500730016034500690042006F00748B
:107130000042006F00610072006400C67009710DAA
:0371400071257145
:0C714400D9CFE6FFDACFE6FFE1CFD9FF9C
:10715000E2CFDAFFFB0EDBCF45F0FC0EDBCF46F0D3
:107160000001800E46141AE1FB0EDBCFE9FFFC0E96
:10717000DBCFEAFFEECFF3FFEDCFF4FFEE2A000EF8
:10718000EF22F3CFE9FFF4CFEAFFFD0EDBCFEFFFF5
:10719000EF50466AF36E46C0F4FF10D0FB0EDB5092
:1071A000FE0806E1FD0EDBCFE6FF9FEC39F005D0CF
:1071B000FD0EDBCFE6FF0DEC08F0E552E552E5CF22
:0871C000DAFFE7CFD9FF12004E
:0871C80037503C02F3CF33F015
:1071D000F4CF34F03D02F3503426000EF420356E27
:1071E00037503E02F3503526000EF420366E3750ED
:1071F0003F02F350362638503C02F3503426F45008
:107200003522000E362238503D02F3503526F45018
:10721000362238503E02F350362639503C02F350A5
:107220003526F450362239503D02F35036263A5076
:087230003C02F3503626120067
:08723800FF0EE124E96EFF0ED8
:10724000E220EA6EEDCFF4FFEFCFF3FFF46607D054
:10725000600EF36404D07B0EF36001D0F39A120049
:10726000F36AF46AFF0EE124E96EFF0EE220EA6E93
:10727000ED6607D02F0EEF6404D03A0EEF6001D018
:04728000F32A1200DB
:0C728400366A356A346A336A200EE76E01
:10729000D8903736383639363A363336343635368E
:1072A00036363C50335C3D5034583E5035583F5094
:1072B000365809E33C50335E3D50345A3E50355AFF
:0C72C0003F50365A372AE72EE4D7120060
:0472CC004F4B0D0A0D
:1072D000000D0A004542427631335F616E645F61A2
:1072E000626F7665204542204669726D77617265EE
:1072F0002056657273696F6E20322E312E35610D06
:027300000A0081
:0E730200C00EF36E00EE00F00E0E01D8120069
:10731000EA6002D0EE6AFCD7F350E9601200EE6A30
:02732000FCD798
:0E7322001DEE00F02DEE00F0F86A329C27EC14
:0E73300037F0B6EC39F072EC36F0FBD71200F5
:02733E00FF0E40
:10734000E350ADBA04D0B06AAC8EAD8A949CADA2C5
:0A735000FED7AE6EF36EF46A120071
:06735A00303132333435FE
:0B7360003637383961626364656600EF
:02736C0012000D
:02736E00FEFF20
:10737000000000000000000000000000000000000D
:1073800000000000000000000000000000000000FD
:1073900000000000000000000000000000000000ED
:1073A00000000000000000000000000000000000DD
:1073B00000000000000000000000000000000000CD
:1073C00000000000000000000000000000000000BD
:1073D00000000000000000000000920F920F920FCA
:1073E000930F930F930F930F930F930F930F930F8D
:1073F000940F940F940F940F940F940F940F940F75
:10740000950F950F950F950F950F950F890F890F74
:10741000890F8A0F8A0F8A0F8A0F8A0F8A0F8A0FA5
:107420008A0F8B0F8B0F8B0F8B0F8B0F8B0F8B0F8D
:107430008B0F8C0F8C0F8C0F8C0F8C0F8C0F00010F
:107440000500010203040506070001020304050606
:077450000702030405060713
:01FFF800AC5C
:01FFF900F710
:01FFFA000AFC
:01FFFB00FF06
:01FFFC0063A1
:01FFFD00F80B
:01FFFE008181
:01FFFF00F110
:00000001FF
